:020000041100E9
:10300000002370B5284C0120636101F035FA40209F
:103010000223FE21254A207401F0B4FA002833D19E
:103020000223FF21224A207C01F0ACFA00282BD198
:10303000204BA2899A4224D1E3891F4A93420CD1A2
:103040001E4B63611E4B2268002A03D1002B01D066
:1030500023CB23C401F084FA70BD1A4A934201D0F5
:103060000023F0E7184B194A1B68934205D9C02288
:103070000421207C920001F0FFFA104B6361144B95
:10308000E1E700232374EBE7CC223820AC21920146
:10309000207401F0F1FA0028F3D10E4B63610E4B5E
:1030A000E3810E4BCFE7C0469463FF1FA063FF1F71
:1030B000A263FF1F5959000083050000D942001187
:1030C0006CBA001182150000B863FF1F871300005F
:1030D00078BA001175430011AAAAFFFF60BA001167
:1030E000F7B5164B0192C318021D002000938823E8
:1030F0005B05D3181B685C1C1AD09CB2402C18D8F6
:103100008D781E0CAC466746CD782D023D43AE420D
:1031100006D1019800280ED110000C70240A4C70C2
:1031200003249BB20733A343D218009B9A42DED3F9
:10313000FEBD4432F9E71000FAE7C046FC0F00007C
:10314000802213B503000324019189B25201073193
:103150009B18A14304305A1A88235B05C3181B68C7
:10316000591C03D190429241104016BD99B240299A
:1031700007D80B000733A343C0189042ECD30020BC
:10318000F3E74430F9E7134B134A1B68126810B594
:10319000FA24934201D81A00F824104BE4021B6869
:1031A0009A4210D813000E4A12689A420ED3013385
:1031B00007D1F823DB029C4203D10A49054808F0F5
:1031C000ABF8200010BDFC24E402ECE7FE24E4028E
:1031D000F7E7C04600C0071100D0071100E0071153
:1031E00000F00711FFFFFF7FF0B59BB015000490C2
:1031F0000391402A00D9A0E006AB59801A80FFF75E
:10320000C2FF0400042816D9002206A9FFF768FFB0
:10321000052810D906AB1B88AB420CD1002D07D076
:10322000514B2A000499C01808F0BEF9002802D1B9
:1032300001201BB0F0BD06AB1D8020000699FFF7F2
:103240007FFF041E7BD1069B0793FFF79CFF802323
:103250005B01C618802307001B039E4201D3F8269A
:10326000F60288235B05F31801931B68013302D033
:10327000019808F0C9F83D49019808F04DF83B1D48
:103280000293331D05938822029B52059B181B68ED
:1032900008935A1C3CD044219AB20091402A04D889
:1032A0000320D11D814389B2009103991B0C8B42ED
:1032B00024D0402A22D80122300008A9FFF710FFAD
:1032C000021E1BD1380008A9FFF70AFF04000428DA
:1032D00031D9009A059B9B1880225201B218934263
:1032E00040D288235B05C118009A09A808F05CF851
:1032F0001D4B009A09A9F01808F076F8009A029B75
:103300009446634402931A4B029AFB189A42BAD32A
:1033100088235B05FC1821680198013907F0FCFF40
:10332000200008F071F8039A07AB5A803000079923
:10333000FFF706FF0400002C03D1002079E70428E2
:10334000FBD988235B05E018069907F0E5FF032306
:10335000EA1C9A4300D16BE7034B0499E01808F08C
:1033600043F865E70424ECE704000011FFFFFF7F4A
:10337000F80F0000F7B505001400402A21D80027F7
:1033800001AE71803780FFF7FEFE042816D93A009F
:103390003100FFF7A5FE042810D93688BC420BD0B7
:1033A000BD4209D0221CB44200D9321C064B92B255
:1033B000C118280007F0F8FF30B2FEBDC04300B2CC
:1033C000FBE703204042F8E70400001137B5042270
:1033D00004000D0001A81649FFF7CCFF02000428E5
:1033E0000BD1019BA34208D3AB4204D0104901A8E2
:1033F0000195FFF7F9FE01203EBD0E4C2368200029
:10340000019308F001F8019920000139019107F0BA
:1034100083FF80235B01E418074B9C42EED104221A
:10342000034901A80195FFF7DFFE0020E4E7C0464D
:103430005555000000C007110000081130B589B0D3
:1034400008F0BAF910226946254808F0DDF8254B46
:10345000009A9A420ED1019B029A0F2B33D8002179
:1034600001240698013B08D2002900D00292029B59
:10347000013331D10023029325E0551CF2D1020023
:103480002100EFE710341022200004A908F0BCF856
:10349000029B013301D1069B0293882304995B05AB
:1034A000C918059B06981A03120B049105928142D4
:1034B00003D02B4201D107F077FF019B013B019321
:1034C000019B002BDED1029B002B03D004930498B8
:1034D0004168084709B030BDE025014C2D03EFE7F6
:1034E0000000011150485936F7B50F490F4B0A68D3
:1034F00004001A4084235B0013430B60030003277E
:103500001033019300252E00112007F0EDFF084B2A
:103510001B683B40AB4002351E43202DF4D1019B7C
:1035200040C4A342EED1F7BD5CF0004000FEFEFFB8
:1035300064F00040802270B5AD4CAE4BD20000214B
:1035400020001C6008F060F92300AB4A88331A6041
:10355000AA4B1A786E23002A00D01133E3620A23A3
:103560002365A74B1878A74BA0630138E361C3B26A
:10357000032B01D810232362A34B37226361C82396
:10358000DB00A36123008C331A60082336210F3A35
:10359000E518E16323646264E9670439251DE9677E
:1035A00025003B26BC352E602500C0352B6025004C
:1035B000C4352A6025000636CC352E602500083E2D
:1035C000C8352E602500D03529602100D4310B602C
:1035D0002100D8310A6021000225E0310D6025006C
:1035E0004221DC35296025001B3EE4352E60250094
:1035F000E8352B602500EC352A6022000525F432E1
:1036000015602200F03211602200183190321160F2
:1036100022009432136023003C2298331A60AF23B7
:10362000DB002360794B2363032805D808F024F9D5
:10363000330235371523636096232100FA225B009D
:10364000A360E360C8332361714BFC319200A36433
:103650000A6062626F4A704DA2627322E2656D3A3F
:103660006265A2650232E5644A60022161669621C4
:103670008900A166626709210022E166A2676749A5
:10368000674A684E2167E2673560032811D808F061
:10369000F3F896089EA61023CDE70E23CBE70C2364
:1036A000C9E720001A259C30056020000735A030AE
:1036B00005602000A83003602300FA20F833800062
:1036C000186023006420A433186023005F38AC33F3
:1036D000186023000338B03318602300C630B433B9
:1036E000186023000020B833186023003825FC330D
:1036F0009D604D4D5A665D644C4D9A64DD61962522
:10370000AD001D624A4D9A675D62F53DFF3D9D62C9
:103710001E25484ADD6618675867D9651966DA6755
:10372000BE23C021444A5B00E250444B4900635031
:1037300004316250C4225200A350FA23E4205B00FB
:103740000432A3500432A3503D493E4A3E4BD1605F
:103750003E49800019503E49E938FF3819503D492B
:10376000043019503C491038D1613C4911633C493F
:1037700051633C4911603C49195019003B48F831EC
:1037800008603B49D16582213A4A89005A501A00A3
:1037900039490832D1671A003849B432116088219A
:1037A000374A89005A501A00364988321160364A21
:1037B000DA6407F0F1FD012007F006FE70BD20007D
:1037C00014259C30056020000435A03070E72000EF
:1037D00010259C30056020000335A03068E72000EC
:1037E0000E259C30056020000235A03060E7C04601
:1037F0000004FF1F6866FF1F6071FF1F2846FF1F40
:103800004A0AFF1F3A07000080C3C9019A0200005C
:1038100050C300006A180000280A0000204E000073
:1038200088130000F009FF1F00400011681000001D
:10383000C4090000DC05000040420F001027000012
:10384000FD1BFF1FFC00FF1F0000FF1F2D2FFF1F90
:103850005532FF1FED30FF1FE11FFF1FFD1FFF1F30
:10386000A921FF1F491FFF1FCD28FF1F952CFF1FF8
:10387000D918FF1FD927FF1F4125FF1F4D25FF1F07
:10388000491EFF1F011FFF1FC11DFF1FF7B50B0CB6
:10389000FF270122009300233C001E001D009446D8
:1038A000019089B262469A401000084018413618CB
:1038B000B6B2FF2F02D1012E00D19FB20098024074
:1038C0001A41AD18ADB2FF2C02D1012D00D19CB22E
:1038D0000133102BE6D10320012E07D1012D04D195
:1038E000019B2401E4191C700138FEBD102EFCD18F
:1038F0000238102DF9D00230F7E710B5064C2378C6
:10390000002B07D10548FFF7EFFD0548FFF7ECFD59
:103910000123237010BDC0462866FF1F3C66FF1FB1
:103920002C66FF1FF0B58BB00D000123019010290C
:1039300036D8FFF7E2FF00231A001B48C15C0133B1
:103940005218102BFAD1023B002A29D0174B184CE1
:103950001F68002306A9E25C1600FA5C56405E541C
:103960000133102BF7D102AA07F09EFF2A0002A90B
:10397000019807F0A9FD07F0D7FE23681B18236004
:1039800007F0D2FE63681B18636007F0CDFEA368E2
:103990001B18A36007F0C8FEE3681B18E360002350
:1039A00018000BB0F0BDC0463C66FF1FC844FF1FA7
:1039B0002C66FF1F0223F0B501245D4D5D4E2B7078
:1039C0005D4B91B01C705D4F0393336804207B7096
:1039D00006F05CFA0023984205D07A78552A02D086
:1039E000332A00D098E03360002006F0CFFC07F0C7
:1039F000B3FCFFF79FFD07F0E7FE1F220124002123
:103A00004F4B10AE1A704F4B1C704F4B19704F4BF1
:103A100019689143163A0A431A6060221968914363
:103A2000403A0A431A6007F007FF07F00DFEC12075
:103A3000FF21474B80001A588A431A50C522920032
:103A400098588843BF3901439950985841490840D4
:103A50008021C9010143802099509958C00509026D
:103A6000090A0143995080213B48490107F0A4FD10
:103A700003232200394901940093394807F044FD9B
:103A80002C22384905A807F08FFC05AC6178207816
:103A9000023406F01BFAA642F8D10021112006F0EC
:103AA00029FB314B314A196803201140A022D20270
:103AB0000A431A608022196892040A431A6019683E
:103AC0002B4A1140802292030A431A60294B2A4A4A
:103AD000934200D8012007F057FC07F04DFE07F095
:103AE000C3FC287807F010FE039B1878C0B207F0DB
:103AF0003BFD07F0A9FE2149042007F09DFD06F0DB
:103B000011FC00F0AFF800F0E5FD00F077FE00F0EA
:103B10000FFA002011B0F0BD00932100174A0420D5
:103B200007F082FC8023DB059C62FFF787FC5BE7E4
:103B30004A0AFF1F34F000402846FF1FC463FF1FDE
:103B4000480AFF1F490AFF1F680AFF1FBCF0004018
:103B500000E100E0FF00FFFF2C46FF1FB058FF1FF1
:103B60002C56FF1F88B9001114F00040FF7FF8FFAA
:103B7000FFFF9FFF6071FF1F0080FF1F3B000108D8
:103B800070B500252849294A29484D6308CA1B05F4
:103B90001B0DED188242F9D10022264B8B63264B78
:103BA00008211A628022254B9205DA67244BDA68D5
:103BB0008A43DA60234A1278012A03D09A6822499C
:103BC0000A409A600121EE242048E40002686C4318
:103BD0008A430260DA6811208A43DA6007F0D4FC75
:103BE000112007F059FC112007F096FE184A200C0E
:103BF0000400642390420AD8FA220023D2009042A3
:103C000005D9144B0A21C01807F066FCC3B2124A4A
:103C10001372124BD4801B78002B04D1104B10214F
:103C2000187807F039FE70BD000005408805054092
:103C300000060540FF01000000F0004004E100E044
:103C40003CF000404A0AFF1FFFDFFFFF0038004042
:103C5000B70B000030F8FFFFAC63FF1FE865FF1FE4
:103C6000E463FF1F002210B51100112007F024FEAD
:103C700010BD0000F8B5002301250826344F354C4F
:103C80003B62E3681120AB43E360E368B343E36066
:103C900007F002FC112007F077FC112007F09CFDD3
:103CA0004023226811201343236080236268DB02D3
:103CB000134363608023A2681343A360A368264A6A
:103CC0001340A3608023A2689B0113431022A360CA
:103CD000236C93432364236C2B43236480235B0076
:103CE0003B62226B1D4B1A402263626B1A40626377
:103CF000A26B1A40A263E26B1340E363E368184AC5
:103D00001340184AE36013682B43136007F0BCFCB0
:103D1000FD21154B154A89005A508023C720626B3C
:103D20005B0313436363E36880003343E360E3684A
:103D30000F4A1D430F4BE5601958114080221202B3
:103D40000A431A50802292051A600B4B5E63F8BD3D
:103D500000F000403CF00040FFFFDFFFEFFFEFFF0F
:103D6000FFFF7FFF003800400000FF1F813B001174
:103D7000FF00FFFF00E100E00000054030B503A8B0
:103D800004880B20002C0ED14968074D087849782B
:103D9000090201430A20A94205D10121200019800E
:103DA000024B1B7A137030BD192A0000AC63FF1F51
:103DB000F7B5150008AA16884A680F4F147852788C
:103DC000120222430A24BA4214D10122DBB2019228
:103DD00000962A0007F0F6F9041E0BD1074B1B686A
:103DE000002B07D068782A780002104342425041E5
:103DF000013098472000FEBD022900003063FF1FFC
:103E000030B5012503790400BFB02B4212D00A4916
:103E1000408806F043FD28420CD06A46074B6946AD
:103E20005B8D55801380064B60881B7A13710022CE
:103E300003F014FE3FB030BD2863FF1F7042FF1F28
:103E4000AC63FF1F10B50549054806F0DDFC0421F1
:103E5000044A054806F09AFC10BDC0462863FF1FBF
:103E6000FFFF0000B4B900117042FF1F10B50248F7
:103E700004F076FC10BDC046013E0011062310B5CB
:103E8000837010330371443B43712A33837144338D
:103E9000C37100230222012103720E4B0270417094
:103EA0001C8881724472197A0273C1729A784273C3
:103EB000DA7882730322C2731A7902745A794274CF
:103EC0000C2282749A79C274DB7903751123C37052
:103ED000152010BDAC63FF1F10B5142007F02CFB9C
:103EE000124B14220021186007F08EFC002007F00E
:103EF0002BFA012007F0A8FA022007F0D5FB0320D7
:103F000003F0D2FE042005F0E7FE052003F010F9CF
:103F1000062003F0DDFD072001F072F9082006F00D
:103F200015FC092000F05CFF10BDC0463463FF1F84
:103F300010B507F0E9FC012007F096FB07F06CFADA
:103F4000002010BD094B10B50400984205D001298E
:103F500004D12000064906F057FC10BD0229FCD10F
:103F6000013904F0BBFB0028F3D0F6E7FEFF0000A8
:103F70005A63FF1F70B50D7A100004AA2C00168832
:103F800010221440154220D1002E20D10A78022A96
:103F900018D14A68517815780E4A0902294391428E
:103FA00005D00D4A914209D01C800A2404E0142255
:103FB0000A491A8007F0F8F9200070BD0C22084960
:103FC0001A80F7E71C800124F6E70824F4E70B24A5
:103FD000F2E7C046F3FF0000F4FF0000AC44FF1F0F
:103FE00090BA001110B504000749084806F00CFC0F
:103FF000074804F0F5FA0020E40704D50721054A34
:10400000054806F0C3FB10BD5A63FF1FFFFF000009
:10401000453F0011F8B90011B442FF1F00B50C4B29
:10402000BFB01A780B4901A800F01AFC6B4680B2A9
:104030005880002809D06A46074B69461B881380C0
:10404000064B0022188803F009FD3FB000BDC046B2
:104050003863FF1F3963FF1F0E43FF1F0E44FF1F0E
:1040600000B50C4BBFB01A780B4901A801F03CFC1D
:104070006B4680B25880002809D06A46074B6946D3
:104080005B8D1380064B0022188803F0E7FC3FB0DD
:1040900000BDC0466263FF1F6363FF1FB442FF1F82
:1040A0000E44FF1FF7B50E00377A1C0008AB110055
:1040B0003D001A8820231D401F423CD13378022B3B
:1040C0003BD173681F785B781B023B431E4FBB429A
:1040D00008D01E4FBB4214D01D4DAB4221D00A2543
:1040E0002800FEBD002A2AD1142C2AD82200F0680C
:1040F00007F05AF9174B1C70012CF1D9FFF7B0FFEC
:10410000EEE7002A1BD1202C1BD82200F06807F014
:104110004BF9114B04211C70104B187807F0BCFBB5
:10412000DEE7E3B20124009201940A00310007F0B7
:1041300049F80500D4E70825D2E70125D0E70B258B
:10414000CEE70D25CCE7C046F3FF0000F4FF0000EA
:10415000022900006263FF1F3863FF1FE463FF1F33
:10416000332310B5040003700A220749013007F019
:104170001BF9064B0F201B681A0AE37222731A0CF4
:104180001B0E6273A37310BDAC63FF1FD463FF1FCC
:1041900030B5012503790400BFB02B4213D00B4981
:1041A000408806F07BFB28420DD06A46084B01A8E8
:1041B0001B881380FFF7D4FF6B46588000226946A6
:1041C000608803F04BFC3FB030BDC0465A63FF1F10
:1041D0000E43FF1F10B5024804F0C2FA10BDC046DE
:1041E0009141001170B5160004AA148805AA15782B
:1041F0004A685078117800022A4A08438018052836
:104200004BD807F039FB03131E29343F0720032C3A
:104210000BD80422121BAA4200D92A0022491A8074
:104220003000091907F0C0F8002070BD0720112CDC
:10423000FBD81222121BAA4200D92A001B491A805D
:10424000EEE707200E2CF0D80F22121BAA4200D94D
:104250002A0017491A80E3E70720032CE5D8042237
:10426000121BAA4200D92A0012491A80D8E7072057
:10427000032CDAD80422121BAA4200D92A000E49C4
:104280001A80CDE70720032CCFD80422121BAA42A4
:1042900000D92A0009491A80C2E700220A201A80A0
:1042A000C3E7C046DCD5FFFF43BA00118063FF1FA0
:1042B00033BA00112EBA001129BA001124BA001124
:1042C00010B50D21024A034806F060FA10BDC04641
:1042D00018BA00112443FF1F37B5002000F0CCF8B6
:1042E000204D214BEA89287C9A422AD1042201A937
:1042F00000F076F9040000F033F9002C30D16B4661
:1043000099882B68C9BA4B432989184A1B145B1832
:1043100053806B46D9886B6849BA89B24B43698927
:104320001B0C5B181248191C1BB2834200DD011CD8
:104330000B0400D5002113889180013313802000E5
:104340003EBD0223002101AA00F01CF96A460400C8
:1043500002230121287C063200F014F90443CAE745
:104360000124ECE79463FF1F83050000AC63FF1F8B
:104370000F27000037B5012000F07EF81F4D0722FF
:104380006946287C00F02CF9041E33D16B461B785B
:104390007F2B2FD800F0E4F86B46D878F023020486
:1043A0001B031A406B469B8815495BBA9BB21A43A4
:1043B0002B68000953432A891B0C9B184B806B46C2
:1043C0005A789B7812031B011A436B6802435343CC
:1043D0006A891B0C9B180B481A1C1BB2834200DD18
:1043E000021C130400D500220B888A8001330B8045
:1043F00020003EBD00F0B4F80124F9E79463FF1FEC
:10440000AC63FF1F0F27000010B50F4C237C002B5F
:104410000CD0382B0BD1012000F02EF8CC22AC218F
:10442000207C920100F028F900F09AF810BD074BAB
:10443000E2899A42FAD1012000F01EF80021207C86
:1044400000F0FAF8F0E7C0469463FF1F8305000010
:1044500010B5084B1A7C002A09D05B69002B06D0E6
:104460009847041E01D0FEF7CBFD200010BD0124AB
:10447000F9E7C0469463FF1F70B5002106000D20C8
:1044800005F06EFE01210C2005F06AFE07F0A4F88D
:104490000400092007F0A0F900222B4B2B4DDA660F
:1044A00061321A6019685B3A9143002E28D0023AB3
:1044B0000A431A60AC4209D10A22DA6107321A6251
:1044C00000221A639A630132DA6370BD204A944273
:1044D00003D11E22DA610532F1E71E4A944203D16C
:1044E0003022DA610632EAE71B4A944203D14322C2
:1044F000DA610832E3E7194A9442E1D16922F7E729
:1045000002220A431A604622AC4203D0104A944267
:1045100004D194225A6106329A61D1E70D4A94423D
:1045200001D1E622F6E70C4A944204D13422FF324C
:104530005A610D32F0E7094A9442C1D1E622520095
:104540005A610A32E8E7C046005000400024F400F7
:104550000048E801006CDC020090D00300D8B805E8
:1045600010B50024064B0920DC6606F095FF2100FB
:104570000D2005F091FD21000C2005F08DFD10BDF2
:1045800000500040F8B51C000023134D0F00EB66EF
:104590006860160007F010F901238022EB66230003
:1045A0002F615200013B08D206F09EFE08200B4A04
:1045B0001168002C03D12000F8BD2A61F2E72B6FAF
:1045C000034203D02B69013C3370013613685B1A38
:1045D000032BEED90124EEE7005000406008FF1FD6
:1045E000002370B5124D1400EB6668600E0007F0F2
:1045F000E3F801238022EB6623005200013B08D23E
:1046000006F072FE08200B4A1168002C03D120002E
:1046100070BD2A61F2E72B6F034203D02B69013C86
:104620003370013613685B1A032BEED90124EEE7D1
:10463000005000406008FF1F002370B50C4C0D00B7
:10464000E366606007F0B8F80123E366256106F0D1
:104650004BFE8020074A80001168636B034205D13E
:1046600013685B1A032BF8D9012070BD0020FCE70A
:10467000005000406008FF1F002370B5134C0E006F
:10468000E3666060150007F097F80123E366266192
:104690000F33626B1A42FCD02B0A23611023626B2A
:1046A0001A42FCD0EDB2256106F01EFE8020084AB9
:1046B00080001168636B034205D113685B1A032BFA
:1046C000F8D9012070BD0020FCE7C0460050004032
:1046D0006008FF1F10B5084CE368002B08D1074B9A
:1046E0001B685B045B0C0A336360054B1B6823602B
:1046F00006F002FFA06010BDD463FF1FC8F00040A9
:10470000CCF0004010B507F057F80F4B996A9A6A41
:104710008A42FBD10D4C6268A0688A18121A531E97
:10472000884200D31300A1602168DA0B52185B04A1
:1047300007495B0C636022600B60064B1A6006F051
:10474000D3FD206810BDC04600F00040D463FF1FB9
:10475000C8F00040CCF0004070B51F4C23793F2BCF
:1047600001D93F2323711D4B22791A701878C0B2EA
:1047700006F072FF18231A491A4A0B801A4913804F
:104780000B805380A379194980200B800C219380E2
:1047900001334B430001191C834200D9011C144B07
:1047A000D18019806379002B11D101336371237A91
:1047B000012B01D8022323726279237A0D485343D7
:1047C0000A21584306F088FE0B4D286070BDA02BCF
:1047D000EDD9A023EAE7C046C863FF1F480AFF1FC0
:1047E0000C44FF1FD445FF1F0A44FF1FB465FF1F81
:1047F0000844FF1F71020000B863FF1FF8B51221C3
:104800000020FEF7E3FD114C011E114D09D10C22D1
:10481000104BC1CBC1C4280006F0F6FFFFF79CFF88
:10482000F8BD0C2220000C49FEF7A4FD0C2802D094
:10483000084B43CB43C40C2228000849FEF79AFDDD
:104840000C28EBD00C220021E5E7C046C863FF1F0F
:104850009463FF1F84BA0011FC0C0000F50C0000EB
:10486000F0B5002504000E0085B0AA4263D04B1CB1
:10487000087801934B788978377909021943F378DE
:104880003F061B040B431F430397207065702528C8
:1048900000D173E012D810280AD806F0EDFF46E5E3
:1048A0002C2C2C87958E2C2C2C2C2C2C2C2CC500B5
:1048B000232800D1A7E0FF23637094E0562857D047
:1048C00010D8332800D199E0552837D02628F2D1C6
:1048D000934B2900132218001D0006F095FFFEF7E8
:1048E0008FFB5AE0722800D17FE0DC2800D1DAE0AB
:1048F000712800D16FE0DB2800D0EFE0042ADAD97C
:104900001025052A05D0551F2A003800711D06F014
:104910004BFD05223100200006F046FD2A0039003B
:10492000601D06F041FD053505E00C2220007D49A3
:1049300006F03AFD0C25280005B0F0BD013A7A4D8D
:104940000C2A13D8002A0AD02800019906F02CFD61
:10495000FFF702FF0C2228007449FEF745FC2900EE
:104960000C22601C06F020FD0D25E4E70C22EBE78D
:104970006D4D6F4B2A0043CB43C2E9E7013A684DC6
:104980000C2A11D8002A08D00199280006F00CFD45
:104990000C2228006749FEF727FC29001322601C1F
:1049A00006F002FD1425C6E70C22EDE70522624958
:1049B000601C06F0F9FC0625BDE712225F49601C69
:1049C00006F0F2FC1325B6E708225D49601C06F0EC
:1049D000EBFC0925AFE77178F72900D96BE7594B54
:1049E000188801F0DDFB0225A5E7574B012A03D00B
:1049F00072781A706270F6E71B785DE72000FFF7A7
:104A0000AFFB050097E7042A04D9504D2F6006F04C
:104A100073FDA860FFF776FE0422039003A9601CD3
:104A200006F0C2FC052586E7494D062A15D906225F
:104A30002800019906F0B8FD00280ED00622019941
:104A4000280006F0B1FC062242492800FEF7CCFB04
:104A500001233D4A11780B43137029000622601C84
:104A600006F0A2FC072566E7931E3B4F1A2B04D8DD
:104A70007378002B09D100F027F9384B39001D78E5
:104A8000601C6A1E06F090FC55E7551E2A0001992D
:104A9000380006F089FC3249AAB23800FEF7A4FBC0
:104AA00000F048F9E9E7022A00D804E77378BFB2BA
:104AB0006370B378A370032A05D0033A390092B229
:104AC000F01CFEF791FB10223900E01CFEF752FCAF
:104AD000C51C002800DB2EE7607084E7DA2800D0D0
:104AE000E9E6042A00D8E6E6082A15D9B3797279EE
:104AF0001B021343F27912041A43337A1B06134341
:104B00003B603B68052231002000039306F04CFC1B
:104B10000422601D03A95AE7FE236370F1E7C04633
:104B20009463FF1F90BA0011C863FF1FFC0C0000C4
:104B300084BA0011F50C0000A063FF1F8063FF1F03
:104B40004845FF1F0E44FF1FC463FF1FD463FF1FB0
:104B50006509FF1FADAC0000C765FF1FC565FF1FDE
:104B6000AEDE000070470000020010B5094B0A32AB
:104B7000094C92B2DA815A8298811882207802F028
:104B800075F90422054B012120781A7006F084FE85
:104B900010BDC046D244FF1F1266FF1F1166FF1FE3
:104BA000013870B5042809D806F066FE0309230809
:104BB00012001E4B0221187806F06EFE70BD1B4BD2
:104BC0000821187806F098FB0022194B1A72F5E7B5
:104BD00080220024164B154D52001A810821287896
:104BE0001A68DC7206F0F8FB2100287806F074FDE4
:104BF000E4E70E4B0821187806F07EFB0D48FFF71E
:104C00003DF90D4B0D4A9B7993800D4A138000228C
:104C1000074BDA720132FF321A810A4B1B78002BE4
:104C2000CCD0094A136006F0F7FCC7E7E463FF1F26
:104C3000B863FF1F1744FF1FC863FF1FD445FF1F42
:104C4000B465FF1FC463FF1F34F0004010B5002996
:104C500004D1042802D10D3005F04CFA10BD00003B
:104C600010B501290ED104280CD10D3005F042FAFF
:104C7000054B1B78002B05D02622044B04485A72A2
:104C8000FFF772FF10BDC046E865FF1FB863FF1F46
:104C9000C40900000300F0B50A4D8E18B14202D1DC
:104CA00052008018F0BD0C782F6824093C5D0F2756
:104CB0001C700C7801313C402F683C5D5C70023305
:104CC000ECE7C0460444FF1F0D22114B10B51A70CB
:104CD0000C23104C10492370093A033B0F486370B2
:104CE00006F062FB2D2301220D490E48A371FFF748
:104CF000D1FF01220C49FFF7CDFF01220B49FFF73D
:104D0000C9FF00220A491000FEF76EFA10BDC04626
:104D1000E465FF1FC565FF1F43BA0011C765FF1F8C
:104D20006709FF1FCC65FF1F6609FF1F6509FF1F8D
:104D3000AEDE000070B5124C132220001149FEF7C0
:104D400019FB114D002817DDAB78002B14D0431C44
:104D50002B7009236B700023001903702878290039
:104D60000130C0B206F048FC297822000139C9B2EE
:104D7000002005F029FC70BDFFF7A6FFEEE7C04656
:104D8000C765FF1FAEDE0000C565FF1F10B5114BE4
:104D90001A781870002A0ED000280BD10E4B1A7802
:104DA000062A07D85423D340DB0703D50B4B1878CA
:104DB00002F05CF810BD0028FCD0074B1B78012BDB
:104DC00002D0033B022BF5D8044B0121187806F0E2
:104DD00063FDEFE7E865FF1F1166FF1F1266FF1F07
:104DE00070B54D4E4D4A4E493070042005F078FAAA
:104DF0000021112005F07EF9112005F05FFAFEF781
:104E0000FFF806F0B9FB032246494748FFF742FF87
:104E10002D24030004221C7044490130FFF73AFF9F
:104E200030230470424D434C437083702E3B062266
:104E300020004149EB87FEF79DFA062813D0200099
:104E400006F04AFD022809D00321200006F0CCFB21
:104E50008D23E3706E3B23711933637106222000AA
:104E60003549FEF7C1F9354B1B68FC335C64FFF72D
:104E700061FF0020FFF78AFF314C324A0121324B9B
:104E80001278207801F0B4FF304A314B12780021BB
:104E9000207801F0ADFF01222E4B1A702E4B5B786B
:104EA000552B31D12D4B3B325A722D4B2D4AAB81B4
:104EB000EA812B826A822021307806F0E5FC01200D
:104EC000404205F0CDFB0120404205F069FCFFF7B0
:104ED000F7F9FEF7B7FF00F09FFC01204042FFF713
:104EE00081F8012006F000FCF72001F03DF90121D6
:104EF000307806F0D1FC307802F014F91A4806F048
:104F00005BFAFEF7B7FE70BD6422184B5B79534322
:104F10001A000A32CBE7C046E463FF1F4D4C001174
:104F2000614C00114845FF1F8063FF1FA063FF1FF6
:104F3000D244FF1F6509FF1FADAC00006866FF1F6C
:104F40001266FF1F3644FF1F1744FF1FE465FF1F53
:104F5000C565FF1FB665FF1FC463FF1FB863FF1F52
:104F6000C4090000CE090000E663FF1FC863FF1FED
:104F7000F8B50A0020230D001A40194251D0534BB6
:104F80001B78002B3CD0FFF7BDFB514B514C524ED0
:104F900099686268737A8A1ADB039A4202D3616065
:104FA000FEF768FE327A217A531EDBB299422AD18B
:104FB000FFF72AFA637A002B1FD0013BDBB2637242
:104FC000002B1AD1454B5B78552B01D106F024FB01
:104FD000E37A002B0CD00023414A424FE37213883E
:104FE000380001331380FEF749FF390006F04CFA10
:104FF000642370795843FFF7B7FD237A0133237296
:1050000020206840F8BD9142D4D300232372FFF7DB
:105010001FFA344F3800FEF731FF390006F034FA3A
:10502000C8E70BB2002B0ADA2F4B187806F07CFC8D
:10503000002801D006F080FB80200002E1E7022476
:10504000214206D0234B01201A72FFF79FFE200059
:10505000D7E70B071BD5FFF755FB1D4B1D491E4C12
:1050600098684A68637A821ADB039A4202D34860DE
:10507000FEF700FEFFF7ECF9FFF7C6F900F0E6FBDC
:105080002368DB0701D5FFF7A5F80820B9E710244E
:10509000214206D00D4B1B78002BD8D1FEF7E6FE3F
:1050A000D5E70124214209D0104800F06DF806F040
:1050B000B3FB2100112005F01DF8C8E70424080007
:1050C000204021429ED0FEF7A9FFC0E7E865FF1F00
:1050D000D463FF1FB863FF1FC863FF1FC463FF1FB4
:1050E000AC63FF1F1744FF1FE463FF1FFC43FF1F58
:1050F000F0B51B4B1B4F1B883A8804001A4E1B4D02
:1051000085B09A420DD832889A420AD3184B1A8831
:105110002B889A4205D1174A174B12881B889A424E
:105120001BD0052001F076F83B8802AA1380338853
:10513000019053802B88114D93800F4B02A91B883F
:10514000D3800F4B2A78188802F092FD0D4B08216E
:105150002878019A1C7006F007FC05B0F0BDC04627
:10516000B265FF1F0C44FF1F0A44FF1FB465FF1FF9
:10517000B065FF1FAE65FF1F0844FF1F1266FF1FCB
:105180000E44FF1FAC65FF1F13B50C4B1C78002CA1
:1051900011D1002801D00A4B18600A4A0A4B117835
:1051A0000A4A10780A4A01920A4A0092002205F03F
:1051B00003F9200016BD1124FBE7C0461166FF1F4E
:1051C000A865FF1F1066FF1F0066FF1F1266FF1F06
:1051D000EC65FF1FF065FF1F10B5064B12201B7812
:1051E000052B06D1044B13221988044B187801F0C3
:1051F000EDF910BD1166FF1F0E44FF1F1266FF1F61
:1052000010B500240122114B52421870104B1C7033
:10521000104B1A8001F086FF04220F4B21001A70F8
:105220000E480C3206F028F9102221000C4806F036
:1052300023F907220B4B1C600B4B1C700B4B1C7093
:105240000B4B1A700B4B1C7010BDC0461266FF1F33
:105250001166FF1F0E44FF1F1066FF1F0066FF1F31
:10526000F065FF1FEC65FF1FC465FF1FC365FF1FCF
:105270001044FF1FC265FF1FF8B5174C06002578C4
:1052800006A814240078052D23D1B41F134FA5B20E
:105290001824BD421DD88D1FADB2BD4219D8FA25C4
:1052A0006D00AA4215D21D000D4F0A3DADB2BD42A0
:1052B0000FD80C4C26800C4C21800C4900240A800D
:1052C0000B4A1380FFF714FF0A4B0421187806F0ED
:1052D00013F82000F8BDC0461166FF1F790C0000CE
:1052E000750C00000C44FF1F0A44FF1FB465FF1F2C
:1052F0000844FF1F1266FF1FF0B50BB20D0089B006
:10530000002B00DB70E1A44E307806F00DFB041E8C
:1053100050D00378A22B00D122E1D02B1AD0912BB0
:1053200045D143780E2B42D19C4B82889A423ED184
:105330009B4A83681278052A39D1032018567F28A2
:1053400035D0984B1B68002B31D05B68002B2ED0DA
:1053500098472CE08078072829D806F08DFA042891
:10536000183F3F74A8D86378002B0CD101218C4BD7
:1053700019708D4B1A78002A5BD08C4B307801F075
:1053800037FD002855D00722854B1A7051E061780F
:105390000029F8D1E378002B11D0854A854B12788B
:1053A000307801F025FD60706378002BEBD1200090
:1053B00006F0C2F980200002684009B0F0BD784BC9
:1053C0001B78022BF3D00121307806F075F8002805
:1053D000EAD10121307806F05FFAE5E76378002B27
:1053E000D1D16F4F032807D13B78052B02D1013370
:1053F0003B701EE00223FBE76F4B1A886F4B029352
:10540000002A0BD01B78002B03D00121307806F046
:10541000ABFA3B78062B04D1013BE9E7029B1A70FB
:10542000F7E7042B41D10121029B3078197006F077
:1054300033FA5C4B1B68002BB9D01B68002BB6D02D
:10544000574A107884E76378554F002B27D10622FE
:10545000211D5B4805F0A8FF62895A4B5A491A8002
:10546000A2895A4B1A80E3890B800521397058496B
:105470000A80584A1380228A574B1A80574B1B7850
:10548000012B09D11F2000F0C5FEFA2292004243F1
:105490000421307806F068FA0022484B75E7312B7A
:1054A00000D070E70022454B1A700323A0E70622C4
:1054B0000021434805F0E0FF0023454A0421138002
:1054C000444A30781380444A138005F015FF0821C0
:1054D000307805F011FFA379083B5A425341304A16
:1054E00003331370304B1B78002B06D0334B3078CE
:1054F0001A78002A06D001F0B9FC0122314B524241
:105500001A8096E70121197006F0C6F9F5E708211F
:10551000307805F0F1FE6378002B00D047E72C4B84
:105520002D4F0293E388029A04211380294B30788F
:1055300003932389039A138063893B8005F0BCFFA2
:10554000002800D033E7264B1B68002B00D12EE744
:10555000039902983A88098800881B68984726E7CB
:105560004379132B00D022E70389012B0AD11D4B6D
:105570001B78022B06D10821307805F0BDFEFFF71D
:105580002BFE14E7052000F045FE082102003078CC
:1055900006F0EAF90BE7C0461266FF1F051400008B
:1055A0001166FF1FA865FF1F3644FF1F1744FF1F2A
:1055B000E465FF1FC565FF1FE665FF1FE865FF1F68
:1055C000B765FF1F0E44FF1FBE65FF1FC065FF1FAD
:1055D000B265FF1FB065FF1FAE65FF1FB665FF1FF9
:1055E000A465FF1FAC65FF1F8020C001014200D0F1
:1055F000E2E6CB0731D5324B1B78002B1DD0314E64
:1056000005AC3378052B1AD1023B23702E4B2100B9
:105610001B7823722D4B1B7863722D4B187801F089
:105620008BFB002809D007202A4B30701B68002B09
:1056300003D01B68002B00D098470120BCE60E2049
:10564000254B06221B7825492370254B1B78637058
:1056500002ABC01805F0A8FED8E7022308001840E6
:10566000194209D0174B1B78052B03D11D4B188805
:1056700006F02AF802209FE60424214203D0FFF717
:1056800037FD200098E6082308001840194200D191
:1056900093E6154B1C78012C03D0022C0DD008206A
:1056A0008AE6124B124A134913481B88128809884C
:1056B00000880094FFF7E0FDF1E7FFF78DFDEEE7CE
:1056C000E865FF1F1166FF1F1044FF1FC265FF1F23
:1056D0001266FF1FA865FF1FC465FF1F1144FF1F4F
:1056E000C365FF1F0E44FF1FAC65FF1F0844FF1F6B
:1056F000B465FF1F0A44FF1F0C44FF1F10B502A82A
:1057000004880B20002C10D14968087849780902D8
:1057100001430C48814209D1022119800A4B598862
:105720001170DB7800205BB2537010BD074C0A206B
:10573000A142FAD102211980034B998811705B793B
:10574000F0E7C0466E2A0000AC63FF1F6F2A00001E
:10575000F7B5150008AA16884A680F4F14785278D2
:10576000120222430A24BA4214D10122DBB201926E
:1057700000962A0005F026FD041E0BD1074B1B687E
:10578000002B07D068782A7800021043424250412B
:10579000013098472000FEBD022900002466FF1F4B
:1057A00030B5012503790400BFB02B4227D015493D
:1057B000408805F073F828420DD06A46124B6946BE
:1057C0005B8D138002235380104B5B88938060882D
:1057D000002202F043F90E49608805F05FF8C00727
:1057E0000DD56A460B4B69461B88138002235380F4
:1057F000064B9B8893806088002202F02FF93FB00F
:1058000030BDC0461C66FF1F3844FF1FAC63FF1F3E
:105810001466FF1F9244FF1F10B5074C0749200074
:1058200004F0F2FF2000064904F0EEFF0721054ACC
:10583000054804F0ABFF10BDFFFF00001C66FF1F12
:105840001466FF1F10BB00113844FF1F10B502483B
:1058500002F086FF10BDC046A15700110200F0B54E
:1058600001270A480A4E51188B1A002B00DCF0BDA4
:10587000082415784308684038404000805B013CAC
:1058800058406D08002CF5D10132EDE7FFFF000014
:105890002ABB0011F0B500250F269D4200DBF0BDAC
:1058A0004C5D070944403440A400A05801357840BD
:1058B000F3E70000F0B589B06A460D000B000F2732
:1058C000110010351C780133260024093E40167063
:1058D00054700232AB42F5D12023024AFFF7DAFFBF
:1058E00009B0F0BD30BB0011F0B54E780B7889B02F
:1058F00036020C00170001901E43012A61D9954B16
:105900009E4200D877E001339E421CD1062A17D16F
:10591000CA788B7812021A430B791B0413434A7915
:1059200012061A438C4B5A6100221A705A808B4A15
:105930005A608B4A9A608B4ADA60002009B0F0BD49
:1059400088225205EEE7884B9E423CD182498B78F3
:10595000002B00D0F6E00C2A31D10F22A37893431C
:10596000E278120213432279120413436279120679
:1059700013434B60E279A07912020243207A0004BB
:105980001043627A12060243CA60E27AA07A1202D7
:10599000024376484A81834208D804236E49142280
:1059A00001980B7005F000FD1420C7E71201D21812
:1059B00089235B059A42F0D801238B70BDE7022A48
:1059C000FAD00523EAE76A4A01239642E6D1FFF7B7
:1059D00003FC052F0CD9E378A2781B02134322792C
:1059E00012041A4363791B061343624A039313603C
:1059F00005F012FEA1E7584D2B78002B9DD1AB7816
:105A0000002B00D1A0E02B8901339BB20093B3425D
:105A100000D091E0132AD4D9CF7C8B7C3F02122195
:105A200020001F43FFF71AFF874200D08EE0002EB0
:105A30003DD1E378A2781B0213432279E96812046E
:105A40001A4363791B06134303930A228B4212D134
:105A5000FF23A370E370237163716B89002B09D15D
:105A6000E37B227C1B0212041343A27B13431B091A
:105A700001336B8100226B89002B8ED0002A67D105
:105A8000686837013818000B6B690003039098426F
:105A900005D9686105F0B8FCEB780133EB706868F4
:105AA0001022A11C381805F09FFC2E8145E76F8954
:105AB000009A7B1E9BB293423AD1E278A3781202FD
:105AC0001A43237905A81B04134362796C681206F4
:105AD0001A43EB6800920392211D0C22049305F0F7
:105AE00063FC0120260004A940421036FFF7E2FEC5
:105AF000013F012F17D1009A0B232861824200D069
:105B00004CE704221C49200005F06EFC042203A986
:105B1000686805F001FDE968039AFF23914200D10E
:105B20003CE7F73B3AE73100FFF7C4FE1036DFE70A
:105B30000923B742A4D831E7009BB34200D9FCE661
:105B400007232BE7022329E7032327E7062325E77B
:105B50000A2323E7FFFE0000AC44FF1F00000111F1
:105B6000FFFF00005048593601FF0000FFFF001101
:105B700002FF000034F00040B844FF1F10B5034C92
:105B80000B000122210000F06BFA10BD3D5D0011F9
:105B90000B8870B506000D000224162B11D92B00BE
:105BA0000322094900F05CFA041E0AD1074B2A8837
:105BB0001B88191C934200D9111C300089B200F0D7
:105BC000EFFA200070BDC046695D00118266FF1FBC
:105BD00010B54A780400013A0B000220012A07D8C8
:105BE0000A78002A04D005222000024900F038FA81
:105BF00010BDC046975D00110A7810B50B00040077
:105C00000220002A04D007222000024900F028FACE
:105C100010BDC046435E00110A7810B50B000400A9
:105C20000220002A04D009222000024900F018FABC
:105C300010BDC046A95E001110B5034C0B000B222D
:105C4000210000F00DFA10BDD95E001110B5034C13
:105C50000B000D22210000F003FA10BD4B5F001174
:105C600010B5034C0B000F22210000F0F9F910BD14
:105C7000A55F00110A7810B50B0004000220002A6D
:105C800004D011222000024900F0EAF910BDC046FC
:105C9000B55F0011002310B51322190000F0E0F9E0
:105CA00010BD000010B5034C0B001722210000F0BE
:105CB000D7F910BD07600011002310B51922190093
:105CC00000F0CEF910BD000010B5034C0B001B22F4
:105CD000210000F0C5F910BD41600011F7B58489BD
:105CE0000D0006000121002C22D000238268D3562B
:105CF0001778002B1EDA0C2C1AD90C3CA4B21319FD
:105D000040880093230002F086FE431E9841013034
:105D10007B06DB0F6B703F23013C1F40A4B2287051
:105D2000AF70AC80002C07D0B3680133AB600021AA
:105D30000800FEBD0020EBE7AC60F8E70B780370CD
:105D40004B8843704B881B0A83700B79C370042007
:105D500070470420022B06D10020537811781B02D3
:105D6000009A0B43138070470B8803700B881B0A43
:105D70004370022070470420009983420AD153786F
:105D800010781B0203430B80D37890781B020343E7
:105D900000204B807047F8B50D004B78012400219E
:105DA000461C03702B788B4201D82000F8BD6B781D
:105DB000B01C4F1C012B10D1890069184B8802229E
:105DC00033704B88B9001B0A7370691805F07CFBAF
:105DD00004360434A4B2F9B2E4E7122359436B1831
:105DE0005A88043132705B8810221B0A737069185C
:105DF00005F06AFB12361234ECE770B5049D14000E
:105E00001E00052B01D8042070BD637812781B0298
:105E100013432B80E378A2781B02134302226B808A
:105E20002A71211D681D063E05F04EFBB2B22A8183
:105E3000F02AE8D82800A11D0A3005F045FB002013
:105E4000E2E7002310B50A789A4201D8900010BD0D
:105E50009A008A185488013304705488DBB2240AEB
:105E60004470948884709288120AC2700430EAE701
:105E700010B51100029C062B04D004201022142B14
:105E800001D010BD022222714B7808781B02034317
:105E90002380CB7888781B02034363800431601D24
:105EA00005F012FB0020ECE710B50C788B7804317C
:105EB0005C43E4B203702200013005F005FB601C76
:105EC00010BD0420022B06D10020537811781B024C
:105ED000009A0B431380704710B50C000A880231FA
:105EE00005F0F2FA208810BD70B504000D0004988A
:105EF0001100012B01D8042070BD167852781202CF
:105F0000324302800200F83255701470E825002CEC
:105F100000D10C35023B9AB24280AA42EBD8023142
:105F2000043005F0D1FA0020E6E70420009983420E
:105F30000AD1537810781B0203430B80D3789078F2
:105F40001B02034300204B80704710B50C000A88E9
:105F5000023105F0B9FA208810BD000070B50121AA
:105F60001E000420049C0E400B4218D1CB40DDB231
:105F70008D4214D90A49DBB2098899420FD3230014
:105F8000F6331D703300580011184978165C090269
:105F9000314301332152D9B28D42F4D8002070BD73
:105FA000CC44FF1F10B50C000A88023105F08CFAB2
:105FB000208810BD10B50C788B7804315C43E4B2B6
:105FC00003702200013005F07FFA601C10BD10B58F
:105FD00011000298032B01D8042010BD14785278C8
:105FE000043B120222430280CA788C7812022243B8
:105FF00042809AB28280F22AEED80431063005F04F
:1060000063FA0020E9E710B50C000B8803700B88D9
:106010001B0A43704B8883704B881B0AC3708A88A5
:106020000430063105F050FAA088043080B210BD6B
:106030000420012B03D100201378009A13707047BD
:1060400010B50C000B8803700B881B0A43704A883C
:106050000230043105F038FA6088023080B210BD99
:10606000F0B589B003931E4B029242000700D05A4C
:10607000019102F020F81325061E2DD0029B012469
:106080000370019B002B04D0001903999847001955
:1060900084B26B461B7A5BB2002B0FDA10213800FA
:1060A00002F01CFB1925002813D130003219E1B28F
:1060B00002F066FC051E0CD10C34A4B2042304AA21
:1060C000380005A993800696948101F0AFFD051E66
:1060D00002D0300005F048F9280009B0F0BDC046F4
:1060E0008066FF1F70B505000C0000280CD0002052
:1060F000814209D010222000044905F0E5F9012071
:106100002B7823736B78637370BDC04670BB00112E
:10611000F0B506000D0017001C0085B002291BD049
:106120000020102907D1022B07D0102B03D115E036
:106130000020102C08D005B0F0BD69463800FFF7EC
:10614000D1FF2A0069460BE069463000FFF7CAFF1D
:1061500022006946380004E0022BE9D12A00390008
:10616000300005F0E1F9E6E7031CF72800D9F72332
:10617000032008499AB2013A0B80D317034006491D
:106180009B189B100B80D30F04499B185B100B804E
:106190007047C046D044FF1FCE44FF1FCC44FF1FB2
:1061A000034B1B888B4202D3024B4000C152704705
:1061B000D044FF1F8066FF1F014B4000185A7047F4
:1061C0008066FF1F1722014B1A8070478066FF1FF1
:1061D00070B505000E2005F02FF9041E13D0D02352
:1061E000037000230622837007494570033005F0D1
:1061F0006BF9064B2100DA8A62811B7E2373044B04
:10620000187805F0C9F970BD9C66FF1F8C66FF1FEA
:106210002045FF1F262803D8024B4000C05A704774
:106220000148FCE7D244FF1FFFFF000070B50600E5
:106230000C00094D1C220021280005F01DF9074B18
:106240001E70074B1C7005F06FF80123002801D069
:10625000002312202B7070BD8C66FF1F2045FF1F8E
:10626000AD66FF1F70B505000D4C0800E260A1602F
:1062700010220021656005F0FFF9012803D11021EB
:10628000A06802F058FD10220021280005F0F4F962
:10629000012803D11021606802F04DFD70BDC04699
:1062A0008C66FF1F70B5041E05D1002903D006229D
:1062B0000D4805F009F90D4B1D78012D11D1002C69
:1062C00005D102221A7005F097FA280070BD00224D
:1062D0001A70074B1B78FF2BF7D02000FFF778FFD1
:1062E000F3E70025F1E7C0469C66FF1F8C66FF1FA1
:1062F0002045FF1F030010B5002801D1002010BD6C
:1063000000780B4A002803D15988D1821B79137673
:106310001378022BF2D10023984200D1033313707B
:10632000044B1B78FF2B01D0FFF752FF0120E6E75B
:106330008C66FF1F2045FF1F002911D000280CD0BC
:106340004B79012803D140225242134303E03F22FC
:106350001340032802D001204B7170474022F4E71C
:106360000800FAE770B5094D0100287800280BD025
:10637000074C0622200005F0A7F821002878FFF737
:10638000DBFF200005F068FA70BDC046AC66FF1F59
:106390008666FF1F00290AD0012808D13F224B79C9
:1063A0009343C02B03D0403B5A425341981C704743
:1063B00070B5174D06002B78FF2B15D00A2005F07D
:1063C0003BF8041E10D0D0230370C83B8370114BE0
:1063D00011491B784670C3700622043005F074F82A
:1063E0002100287805F0D8F80C4B1B78012B0DD133
:1063F0000B4B1B68002B03D09B68002B00D09847E9
:10640000084B04211878084A04F0E6FF70BDC04626
:106410002045FF1FAC66FF1F8666FF1FA866FF1F93
:10642000D466FF1FD866FF1F60EA0000014B986822
:106430007047C0468C66FF1F014BDB6818687047C9
:106440008C66FF1F074B10B5DA68136801331360C1
:10645000054B1878FF2803D08021C90105F01CFAEC
:1064600010BDC0468C66FF1F2045FF1FF7B50E000C
:1064700002F0C8F8051E1CD00E4B06621F78002FD4
:1064800000D10778AB791020019304F0D5FF041EEA
:106490000FD0D0230380C73B8370019BE91DC370DD
:1064A0000622043005F010F821003800E66005F0FF
:1064B00073F8F7BD1E45FF1F014B18787047C046A3
:1064C000AC66FF1F054B002805D1054B1A78054B1C
:1064D000002A00D1014B18007047C0469C66FF1F80
:1064E000AC66FF1F8666FF1F014B58687047C046A9
:1064F0008C66FF1F024B1868431E9841C0B270475C
:10650000B066FF1F421E03000120152A03D9FF3B7E
:106510005A425341D8B27047F0B51C0000230E0018
:1065200085B0039002920B70029A934201D300202F
:1065300019E0E55C5A1CD2B2002DF8D0029851192E
:106540008142F4DC0233DFB2A35C18000193FFF751
:10655000D9FF002807D0013D019A0399EBB23370AF
:106560008A4202D1E01905B0F0BDDB19DBB2DBE7EE
:1065700010B50C0002F09EF803001220002B03D08F
:106580002100588805F0C8F810BD000070B50E4D08
:1065900084006359002B15D0186A002801D005F03B
:1065A00003F92B59586A002801D005F0FDF82B5942
:1065B000986A002801D005F0F7F8285905F0F4F89A
:1065C00000232B5170BDC046BC66FF1F1C4B70B52D
:1065D00004000E00150099420AD11A4B1B68002BCB
:1065E00001D1122070BD1B68002BFAD09847F9E743
:1065F000154B994215D1134B1B68002B0AD01B6811
:10660000002B07D09847002804D1104B1C70104B6A
:106610001D70E7E729002000FFF7AAFF0028E1D15D
:10662000F3E7080001F0EEFF0028DAD0037803203A
:10663000A342D7D12900300005F06EF8D2E7C0465A
:10664000FEFF0000B866FF1FFFFF0000B566FF1FDA
:10665000B466FF1FF7B50400808801F0D3FF002562
:10666000A84203D00578A08802F008F81C4E3378C1
:10667000002B1FD0AB421DD11A4B28001978FFF711
:1066800077FF002818D000233370A3790820A7785B
:10669000A688019304F0D0FE011E0DD0D023037014
:1066A000CA3B8370019B477086808371280004F089
:1066B00073FF01E0002DE8D1A0880B4B8200D35876
:1066C000002B01D0FFF762FF1721A088FFF768FDBC
:1066D000A08801F027FDA08801F0FEFDF7BDC046AF
:1066E000B566FF1FB466FF1FBC66FF1FF0B587B01D
:1066F0001D000CAB1B88070001930DAB1B881420F9
:1067000002930EAB1B88160003930FAB1B880091FE
:10671000049310AB1B88059304F08EFE041E1AD060
:10672000D0230370CB3B47708370C67006222900CC
:106730000430002D11D004F0C7FE019B21006381BD
:10674000029B0098A381039BE381049B2382059B0A
:10675000A37404F021FF07B0F0BD04F08DFEECE758
:10676000F7B5009308AB1B8807000C200D0016003E
:10677000019304F061FE041E13D0280001F042FFD3
:1067800000280FD00078D0232370C93BA370009B52
:1067900021002381019B6770A580E680638104F05E
:1067A000FBFEF7BD014B1878EDE7C0462045FF1F03
:1067B00013B5040064890389C2888188C078009475
:1067C000FFF7CEFF13BD000010B5044C2068002871
:1067D00003D004F0E9FF0023236010BDC066FF1F53
:1067E000A122F0B5818892004A43384B384F1B688C
:1067F00004009B189D2292009B18827989B01A6030
:106800003B68002B5FD01D78324B1B68002B04D0F7
:106810005B68002B01D00020984726000836310025
:10682000E079FFF7B7FD237DE0710200E078049383
:10683000638A29000393238A0293E3890193A3883F
:1068400000933300FFF752FFE378002B0BD1E2896E
:10685000A379A18802920196E27928000092012290
:1068600001F0DAFEE0703B68002B20D0FFF7ACFFB0
:10687000194D287800281AD0184B1978FFF778FEA0
:10688000002814D02B78E67808200793A78804F016
:10689000D3FD011E09D0D0230370CA3B467083701C
:1068A00087808671079804F077FE00232B701721EC
:1068B000A088FFF775FCA08801F034FCA08801F0E7
:1068C0000BFD09B0F0BD064B9DE7C0463409FF1F24
:1068D000C066FF1FD466FF1FB566FF1FB466FF1FAB
:1068E0002045FF1FF8B5070008000E0001F08AFEE2
:1068F000041E18D02620FFF78DFC051E00D1257838
:10690000062004F099FD041E0DD00021062204F09B
:10691000B3FDD0232370C23B21006770A370A68013
:10692000E8B204F039FEF8BDF0B585B001930AABCA
:106930001B78070002930BAB1B7808000D00009238
:10694000039301F05FFE061E22D0102004F074FDB8
:10695000041E1DD01022002104F08EFD2620FFF71A
:1069600059FC002800D13078D0232370C13BA3709C
:10697000009B21002372019B67706372029BA580BC
:10698000A372039BC0B2E3720C9BE36004F004FEAD
:1069900005B0F0BDF7B50D00019001F033FE071E04
:1069A00020D00E2004F048FD041E1BD02620FFF747
:1069B00031FC061E00D13E78D0232380C53B062241
:1069C000A370F91DE01C04F07FFD019B2A00638188
:1069D0000123DD401A401D40210022736573F0B28F
:1069E00004F0DAFDF7BD0000F0B585B002901000AC
:1069F0000D0017000A9E039301F004FE041E31D01F
:106A0000029B002B2ED1039B02795B0724D5122316
:106A100013430422002E08D10B99002905D10C99AB
:106A2000002902D10D9900291AD01A430D9B227119
:106A3000002B00D0C9E0002E00D1CFE0002D00D007
:106A4000CCE0606A002801D004F0AEFE1C213000CA
:106A500004F07AFD606205E002239A430E33D7E723
:106A600093432371654BBA00D458002C00D1AAE09F
:106A7000002E10D0236A002B03D11C2004F05CFDF3
:106A800020625E4BBA00D358186A002803D01C223B
:106A9000310004F019FD0C9B002B12D0574CBB00A9
:106AA0001D596B6A002B03D1162004F045FD686266
:106AB000BB00E358586A002803D016220C9904F052
:106AC00003FD0D9B002B11D04C4DBC006659B36AE1
:106AD000002B03D1142004F02FFDB0622B59986ACB
:106AE000002803D014220D9904F0EEFC380001F0C8
:106AF00089FD051E67D0414BBA00D358002B62D0E8
:106B00001A6A3420002A00D11C389A6A002A01D05F
:106B1000143080B20B9A002A01D01C3080B25B6A1C
:106B2000002B01D0163080B204F086FC041E4AD03F
:106B30001822002104F0A0FC2620FFF76BFB019037
:106B4000002801D12B780193D0232370029B2000D1
:106B500063700A23294EA370039BBD00A371AB5938
:106B6000A780196A1830002905D01C22A06004F003
:106B7000ABFC200034307359996A002907D0030018
:106B800014221433E060029304F09EFC02980B9BE5
:106B9000002B08D003001C221C330B9920610293A8
:106BA00004F092FC02987359596A002903D0162206
:106BB000606104F089FC6B462100187904F0ECFC5C
:106BC0003800FFF7E3FC05B0F0BD10220D9B0D99D6
:106BD0001B69A018236204F077FC2CE70B9B002BA9
:106BE00000D13FE7012D00D03CE7606A002801D0CA
:106BF00004F0DAFD1C210B982AE7C046BC66FF1F93
:106C000010B5044C2068002803D004F0CDFD00230B
:106C1000236010BDB066FF1F0B4B07B51A68002A32
:106C200001D100200EBD6946531C012012780731A6
:106C3000FFF772FC0028F4D00278012310001840FE
:106C40001A42EED0EEE7C046CC66FF1FF0B51F4FEC
:106C500001203B6887B0002B25D09B78059300F07E
:106C6000B3FB002821D00A20FFF7D4FA04000B2040
:106C7000FFF7D0FA164B05001E78731E9E413B6845
:106C8000F6B2191DD878FFF757FB3B682900DA7A6E
:106C9000043303929A79019302920090330020000A
:106CA000059A04F049FE07B0F0BDFFF7B5FF0028D4
:106CB00005D00620FFF7AEFA04000720D8E7082029
:106CC000FFF7A8FA04000920D2E7C046B066FF1F0C
:106CD000AC66FF1F70B50A4E040033780D00FF2B21
:106CE0000DD0042004F0A8FB011E08D0D0230370AF
:106CF000CE3B45708370C470307804F04DFC70BD9D
:106D00003045FF1F70B5040006200D0004F094FB11
:106D1000011E0AD0D0230370CD3B8370054B447015
:106D20001B688580187804F037FC002C01D0FFF731
:106D300067FF70BDB066FF1FF8B5264F06003B68C1
:106D40000D001124002B05D10522234B1B78134283
:106D500002D112242000F8BD204A10241268002A13
:106D6000F8D01278002AF5D0DB0719D52B789A1EB7
:106D7000012A1AD80C2004F0DFFB13243860002805
:106D8000E8D000230A22437029000670023004F084
:106D90009BFBFFF75BFF041E0AD0FFF731FFD9E72B
:106DA00000F012FB0028E1D1E4E7002BE2D0D0E7AD
:106DB0000B4B1B78032BCDD11D20FFF72BFA094B72
:106DC00018800028C6D0084B04211878074A04F020
:106DD00003FBBFE7B066FF1FAD66FF1FCC66FF1F5A
:106DE000AC66FF1FAA66FF1FD866FF1F60EA00009F
:106DF000F7B50193194B14001A78052306000F000C
:106E000012201A4221D0012920D1154B1D68002DD6
:106E10001BD002201F2C18D8002C02D0019B002B65
:106E200013D0104B1F221E706E1C0021300004F086
:106E300023FB01992200300004F046FB31002000C2
:106E40002C70002F06D004F077FAFEBD064B1220FE
:106E50001D68DCE704F0D0FBF7E7C046AD66FF1F16
:106E6000CC66FF1F3045FF1FC866FF1FF8B50F4EE9
:106E700012243368002B17D01B780F3C834213D1A8
:106E800000250B4F0221387804F036FA094B042113
:106E900038781D8004F030FA074B28001D803368D5
:106EA0005C7004F001FB04002000F8BDB066FF1F19
:106EB000D866FF1FC466FF1FAA66FF1F70B50128B2
:106EC00023D11B4C2388002B03D01A4A1578002DA0
:106ED00007D0194B1B68002B02D01878FFF7C6FFAC
:106EE00070BD3B2B02D93C3B2380F9E7134E0221B6
:106EF000307804F001FAFA222388920002215A43E2
:106F0000307804F031FD2580EAE70B4B1B68002B3D
:106F1000E6D00B4B1B785B07E2D5084B02211878B3
:106F200004F0EAF90022024B1A80FFF769FED7E766
:106F3000C466FF1FA866FF1FB066FF1FD866FF1F4D
:106F4000AD66FF1FF8B51E4D2868002803D004F079
:106F50002BFC00232B601B4E3068002803D004F06C
:106F600023FC00233360184F05243B781800204091
:106F7000234221D0154800F02BFA3B78234213D04E
:106F8000202004F0D9FA2860002813D02022002104
:106F900004F072FA202004F0CFFA041E306005D00D
:106FA0002022002104F068FA002004E0286804F0A0
:106FB000FBFB2C601320F8BD00F00AFAF4E7C04692
:106FC000CC66FF1FC866FF1FAD66FF1F2445FF1F6D
:106FD00010B50A4C23681A1E0ED0002808D10130C3
:106FE000587004F061FA002805D02368002B02D005
:106FF0000021FFF787FE0122100010BDB066FF1FC1
:10700000F7B5274E050033680191181E21D05C7832
:10701000244F012C30D1FFF7FFFD002825D02000A0
:10702000FFF7F8F80400412814D91F4B0221187803
:107030001E4A04F0D1F91E4B3C3C1C8002223368EE
:107040005A703B78002B14D128000199FFF75AFEA3
:107050000120FEBDFA2292004243002AEED0124BDC
:107060000221187804F080FCE8E7FFF7D3F802006B
:10707000F3E700233B70EBE73B78002BE8D10320DC
:1070800004F0DAF9011E08D0D0230370CC3B457020
:1070900083703368187804F07FFAFFF7B1FDD7E703
:1070A000B066FF1FA866FF1FD866FF1F60EA0000DA
:1070B000C466FF1F10B51749838802008B4220D099
:1070C00011D815498B4217D0144900205B1899B28A
:1070D000012907D8926811785A425341D8B2FFF774
:1070E000F9FD012010BD0E4A00209B1807229BB21B
:1070F0009A424041C0B2F5E783681878FFF768FF0D
:10710000F0E7836899785A78090218781143FFF7F5
:1071100077FFE7E70A20000006200000F8DFFFFF06
:10712000AFDFFFFF014B18707047C0463145FF1FAE
:1071300010B5064C207001F041FA207804F0CCF82C
:107140000521207800F062FD10BDC046D866FF1F03
:107150000BB273B50D00002B00DBC4E0884B187830
:1071600004F0E2FB041E0ED00378912B0FD0A22B6B
:1071700000D1A1E0834B1878FF2852D0210004F001
:107180000BFA00284DD180200002684076BD43787C
:107190000F2B76D013D8052B70D00E2BEAD1808818
:1071A000794B98422BD8794B98421BD8784B984210
:1071B000E0D1A3681878591CFFF774F838E03E2B2B
:1071C000D8D18378032B74D06CD8012B6ED0022BCE
:1071D000D0D1704B1B68002B23D05B68002B20D0D4
:1071E00098471EE06C4BC0180C28C3D804F0D4FAA2
:1071F0001DC2C2150BC20B0B0B3223C23C00674BE6
:10720000C0180728B6D8664B1B68002B09D01B682E
:10721000002B06D0200098470AE0A3681878FFF7F3
:10722000C7F8200004F088FAADE7A068FFF762F81D
:1072300000289FD0F5E7A3681B78002BF1D0554BB1
:107240001B68002BEDD01B68002BEAD021005548AD
:107250009847EDE74F4B1B68002BE2D01B68002BD3
:10726000DFD021005048F3E7504B1B68002BD8D0EB
:107270005B68002BD5D021004348E9E7FFF7EAF926
:10728000CFE780884A4B984203D04A4B984200D0BF
:1072900070E7464B1B68002BC3D05B68002BC0D047
:1072A0002100D5E7153B012BBBD963E7FFF798FA1F
:1072B000B7E7FFF77DFAB4E73F4B1B78042B07D104
:1072C00000236A4613800179408800F0C5FCA8E7D6
:1072D000364B1B68002BA4D05B68002BA1D00100AB
:1072E000364898479DE7012421420AD0294B1B6864
:1072F000002B04D05B68002B01D0002098470120B0
:1073000043E78B070AD5264B1B68002B04D05B682C
:10731000002B01D020009847022036E704212800E6
:1073200008400D4200D131E7254E3388002B21D093
:10733000013B9BB23380002B1AD1FFF7DBF800280A
:107340000AD0204B1C70164B1B68002B04D05B68C6
:10735000002B01D020009847FFF7C6F8694601F0DE
:1073600001FD6846FEF7FEFF1D20FEF753FF30804B
:1073700004200AE7024B187803F0BEFFF8E7C04686
:10738000D866FF1F3145FF1F0E20000001200000BE
:1073900009100000D066FF1FFEDFFFFFAFDFFFFF19
:1073A000D466FF1F0C2000000B200000B866FF1FF2
:1073B0000D20000013200000AD66FF1FFFFF00003E
:1073C000AA66FF1FA866FF1F10B501F09BF910BD4C
:1073D000014B18607047C046D466FF1F0B88002021
:1073E000162B01D817230420014A13807047C0468A
:1073F0008266FF1F00207047074A03001188814200
:1074000007D091880020994202D1013080001018E5
:1074100070470020FAE7C046E066FF1FF0B58F789E
:1074200006000D00C7B01E2F15D1FFF7E5FF051EA2
:1074300003D10024200047B0F0BD00223B00310002
:10744000C078009200F0B2FB0400A81C00F0D3FB4F
:10745000FF23EB70EEE7264B062403931B78FF2BEC
:10746000E8D0182FE6D87B08224A013BDB000292C5
:107470009A589446002ADDD0029AD3185B68002BF4
:10748000D8D00878002802D14B78012B02D10624ED
:10749000122FCFD107AFAB88697800976446AA68EE
:1074A000A047041EC6D1AB78029A5B08013BDB0003
:1074B000D318390030005B689847041E0BD1AB78B5
:1074C000042BB6D0039A310010782200009700F008
:1074D0006DFB0400AEE76A78002AABD1AA7805A953
:1074E0003B88087130000A704B80FEF747FBA0E72D
:1074F0003445FF1F80BB00111D4B37B50500984276
:107500000BD000290AD1FFF777FF002805D11948D1
:10751000FFF772FF002800D0058037BD01291AD17E
:10752000FFF76AFF041EF8D001235B420380A378B3
:10753000FF2BF2D0FE2B07D00023E078142200931B
:1075400029001E3300F032FBA01C00F054FB012385
:107550005B426380E1E70229DFD1013901F0BEF827
:107560000028DAD12800FFF747FF041EDFD1D4E757
:10757000FEFF0000FFFF0000022210B5074B524241
:107580001A80074801325A809A80DA8000F07EFA29
:10759000044801F025F8002010BDC046E066FF1F3A
:1075A0001D740011F97400110388F7B50400002B55
:1075B00002D102252800FEBD426802211378254829
:1075C0005268FEF7A5FD00282ED0234F01253A88EA
:1075D000002AEFD0802321885B0201259B1A994263
:1075E000E8DC0C2003F0A8FF061E31D03B8822887F
:1075F0009C4600231800019561469DB2491989B245
:10760000AA421BD8002801D062443A8000233000EF
:10761000082208C0210003F057FF104A1368002B0E
:1076200013D100251660C5E76268022113780C4863
:107630005268FEF76DFD0028C7D1BAE760681D01EA
:107640004019418101330198D6E71A001B68E6E72B
:107650001325AFE7EEBB00113245FF1FDC66FF1FAD
:10766000ECBB0011014B18707047C0463445FF1F3A
:1076700014230A0010B51A40194204D00122102127
:1076800001F048F810BD4B06F9D4012088434000B2
:10769000F8E710B514008B0604D50122102101F083
:1076A00039F810BD08230A001A40194202D14BB222
:1076B000002B0FDA102101F02DF8002808D023004C
:1076C000F9331B78002BECD0F8342378012BE8D168
:1076D0000020E6E703208907FAD4E2E7F0B51F00AF
:1076E000184B85B01C68019002910392002C27D1A1
:1076F000200005B0F0BDA5683301ED186B89019A33
:10770000934211D3029A93420ED8002F04D10A9BC0
:10771000002B10D12C00EBE73B002978039A686816
:10772000FEF7F6FC0028F2D10136B6B2A388B342C8
:10773000E1D82468DAE7A3680A9A5B891380E9E74D
:107740000026F3E7DC66FF1F37B50C000A8849887E
:107750000123914217D3002A15D0651D23792A00F1
:1077600002210A48FEF7D4FC102300280BD023790D
:107770006188208800242A000094FFF7AFFF0A23C5
:10778000A04200D0230018003EBDC046EEBB001151
:1077900013B50A0008884988012388420BD80028BD
:1077A00009D00024137905320094FFF797FF0A23CC
:1077B000A04200D02300180016BD13B50A000888A7
:1077C0004988012388420BD8002809D00024137966
:1077D00005320094FFF782FF0A23A04200D0230065
:1077E000180016BDF0B58BB003904A8808880E00CB
:1077F0000123824255D3002853D00023012704AC33
:1078000023700022718813000092FFF767FF051EA6
:107810003ED02078002835D12B78022B18D1677004
:107820006A8983000130E31880005A806968022267
:10783000201803F049FE23780133DBB22370042BB8
:1078400019D93B006889013080B2002BD9D01FE0E4
:1078500002236370122358436A89231804305A8024
:1078600069681022201803F02FFE23780133DBB261
:107870002370002BE5D10C4A6B899B185A42534167
:10788000DBB2DFE76378012BE4D12B78022BC7D082
:1078900022780A23002A04D021000398FEF798F9E1
:1078A000002318000BB0F0BD0100FFFF0F4BF0B537
:1078B00004001868002816D083685D89A54207D89F
:1078C0008288AE18B44203DA12019A18934201D1A9
:1078D0000068EFE71E005F891036A74204D1002937
:1078E00000D00D801800F0BD3300EFE7DC66FF1F0D
:1078F00070B505000C0008880021FFF7D7FF0300D2
:107900000120002B04D022002800197AFFF7C1FEC5
:1079100070BDF7B50C00002501902300F6331B78ED
:10792000AB4201D800200AE06B00E65A002130008B
:10793000E718FFF7BBFF002802D126800130FEBD0B
:10794000017A0198FFF794FE002802D03B8823803B
:10795000F5E70135EDB2E0E710B504000888002135
:10796000FFF7A4FF03000120002B03D02000197AA9
:10797000FFF77EFE10BD0000054B1B68002B01D1F8
:10798000180004E09A6852898242F6D198887047BC
:10799000DC66FF1FF0B50E27002687B0039302AB0D
:1079A000FF183E8005001F4B40891400984207D005
:1079B0002B78013000976A6880B2FFF78FFE0600CF
:1079C00002212B7818486A68FEF7A2FB00280FD026
:1079D0006C892000FFF7D0FF002802D0013C041979
:1079E000A4B2039B002B00D01C80300007B0F0BD78
:1079F00002212B780D486A68FEF78AFB0028E7D140
:107A000002212B780A486A68FEF782FB002807D01B
:107A1000002EDED03B88A342DBD17489013CDFE736
:107A20006C89DEE7FFFF0000EEBB0011ECBB00112C
:107A3000EABB001110B50C00FFF7DEFC03000220CA
:107A4000002B0AD0002C00D023609B781720FE2B3F
:107A500003D00138FF2B00D1002010BD73B50D00FD
:107A600001A904001600FFF7E5FF172805D0002E36
:107A700004D129002000FEF727F976BD012210214C
:107A8000200000F047FE0028F3D0F6E7014B186015
:107A90007047C046EC66FF1F37B56B469D1D010061
:107AA00004000222280003F07FFC2B88B02B0ED1AB
:107AB0002379122B09D12300FF339B78012B06D1A8
:107AC0000121608800F0E0F801E01B2BF8D037BD01
:107AD00010B5054B0421187000F098F8FFF74CFD25
:107AE000FEF770FB10BDC046F066FF1F0020F0B52A
:107AF0000BB20F0087B0834234DA274B187803F0BB
:107B000013FF051E2BD00378A02B25D103AE310027
:107B1000FEF7E4F8041E0BD1B378DB0724D51F4B26
:107B200006341B68002B03D0310068889847040096
:107B3000A868002801D003F017FC002C08D1184ACF
:107B4000039B1340174A934206D0B3781B2B03D0F4
:107B50000121688800F098F8280003F0EDFD8020EE
:107B60000002784007B0F0BD0F4B1B68002B10D00F
:107B7000310068889847041EDAD07378002BD7D17B
:107B8000B27801A90A704B800C716888FDF7F6FF86
:107B9000CEE70624F1E7C046F066FF1FE866FF1F48
:107BA00000FFFF0000011200EC66FF1FF7B5019017
:107BB000822040000D0017001E0003F03DFC040071
:107BC0001320002C12D0B02320002370089BFC222D
:107BD0006770658026710830002B08D0190003F00B
:107BE00073FC2100019803F0D7FC0020FEBD08992A
:107BF00003F042FCF5E710B5041E06D00078FD281E
:107C000003D803F0A9FCFF23237010BD0A1F93B211
:107C100010B504000220032B05D882400020024B3F
:107C2000D1529B189C7010BD1067FF1F0B8870B558
:107C3000043B04000D000220032B0BD8012120007F
:107C400000F04CFD03001420002B03D0290020007D
:107C500000F0DEFB70BD000007B51300034A009280
:107C60000A00012100F02CFC0EBDC046957E0011DB
:107C700007B5019203220092024B0A00122100F084
:107C800049FC0EBD137F001107B56B4601AA118098
:107C90000449D88008780633012802D1190003F07E
:107CA0005BFE07BDF166FF1F0C4B10B5187000237B
:107CB000FF210B4A1380138193819380094A5380DB
:107CC0001370517293819372D174D382137551776B
:107CD00003F052FE00F0FCF910BDC0462067FF1F04
:107CE0001067FF1FF266FF1FF0B58DB06B460020D6
:107CF00003910C229B5E834200DBB0E05D4B187861
:107D000003F012FE051E00D1A4E00378902B00D0F2
:107D10009DE006AF01004688380000F013FA79684C
:107D20000400002900D19CE03B88052B6ED13B89E3
:107D3000032B1CD905AC200000F0A2F86288172A9A
:107D400061D83989131D994231D17968237804317A
:107D50000291D90738D5607800F08EF9071E06D059
:107D6000002303712378012B08D0132B23D0A8689C
:107D7000002800D178E003F0F7FA75E062880299F4
:107D800009A800F0A6F80290380000F08BF909AAC3
:107D90002378387A0192002231000092029A00F092
:107DA00012F9380000F064F9029B002BDFD030009C
:107DB00000F080F9DBE70378032BD8D162880299C1
:107DC00009A800F0D6F8DEE7122B13D1029909A812
:107DD00000F0B5F8021EEAD127498B88002BC6D0E7
:107DE000887909A92378019161780091310000F028
:107DF000EAF8BCE7002302AA93833000617809AA5D
:107E0000FFF72AFFB3E71D4B0993F6E7042B02D0D7
:107E10009A1F012AABD8184A043B9B00995A0029A3
:107E2000A5D0D218907831003A0000F0AEF80028C2
:107E30009DD13B88042B03D001213000FFF724FFA4
:107E4000012C04D1A868002801D003F08DFA280085
:107E500003F072FC8020039B0002434018000DB029
:107E6000F0BD012800D182E701213000FFF70CFFAF
:107E7000EDE7C0462067FF1F1067FF1F01001700D6
:107E80000B7803704B784370CB788A781B021343CE
:107E9000438070470A88030002700A88120A427001
:107EA0000A88012A06D14A8882704A88120AC2705A
:107EB0000420704702208242FBD14A8804309A7025
:107EC0004A88120ADA708A881A718A88120A5A71E4
:107ED000EFE710B50400012082420CD94B780A78F4
:107EE0001B0213432380834206D1CB788A781B027E
:107EF00013436380002010BD022BFBD1CB788A781E
:107F00001B02134363804B790A791B021343A3803E
:107F1000F0E70B8803700B881B0A43704B88837053
:107F20004B881B0AC3708B8803718B881B0A4371B3
:107F3000CB888371CB881B0AC3710820704703006C
:107F40000120082A14D14A780878120202431A80C4
:107F5000CA788878120202435A804A790879120254
:107F600002439A80CA798879120202430020DA809B
:107F7000704710B504000120022A05D100204B787B
:107F80000A781B021343238010BDF8B506001020A9
:107F90000F00150003F050FA04000120002C0ED051
:107FA000A0230C22290023806780201D002D07D0EC
:107FB00003F08AFA2100300003F0EEFA0020F8BD49
:107FC00003F05AFAF6E7F7B51E00009008AB14204C
:107FD00017001D78019103F02FFA041E12D0A2237E
:107FE0000370019B47704380099B057146710C2209
:107FF0000830002B07D0190003F066FA2100009822
:1080000003F0CAFAF7BD099903F036FAF6E737B577
:10801000041E0FD04388002B0CD00025C1881323E9
:10802000007A172201950095FFF7CDFFFF236580A9
:108030006372257037BD000010B50C4904004A88F2
:10804000002A09D08B89002B05D00020CB8A022280
:10805000834201D010BD012213000A2043430020B7
:108060004032C854C81842800472F3E7F266FF1F1A
:108070000023438003707047094B00211A0010B59C
:108080005C88002C06D01C79844203D10A234B4320
:10809000D01810BD01310A330329F1D10020F8E7CF
:1080A000F266FF1F10B50400407A03F055FAFF2373
:1080B000637210BD7047043010B580B203F0FCFA53
:1080C000002803D00421494203F05EFB10BD0000EC
:1080D00070B50025104CA0682580A581A580A84218
:1080E00002D003F041F9A56000250C4C0C4B606DEB
:1080F0001D80230058331D70A84202D003F034F9CC
:10810000656500256068002801D003F02DF9013570
:1081100008340A2DF6D170BDB867FF1F5C67FF1FDA
:10812000AC67FF1F70B5041E09D1054D2880A881DA
:10813000A880A868002802D003F016F9AC6070BDD2
:10814000B867FF1FF0B54B8885B0019300234360EB
:108150000A7905000F00022A00D07BE0CA88032AB2
:1081600017D98B685E7819783602DC78D8790E4397
:1081700099781B7A24021B020C43034353495BBAD0
:108180000B80331D93421ED1042C04D0631F022B9D
:108190000ED9012015E0019A4D4B1201D35A002B44
:1081A00006D00198FFF7BEFF4A4A136901331361F5
:1081B0000421B8682E812C80494203F0E5FA6860FA
:1081C000002005B0F0BD434D042C06D0631F022BE8
:1081D0000FD9EB680133EB60DBE7019A3C4B1201EE
:1081E000D35A002B05D00198FFF79CFF2B69013370
:1081F0002B61374B30000293019B029A1B010193C4
:10820000002301998C468B52130063449C80039396
:108210009E81FFF750FF039B041E986016D0042137
:10822000B868494203F0B0FAFA880100043A200025
:1082300003F04AF90199029AFB888A5A043B9B1879
:10824000029A8B522B6801332B60A2E7AB69013392
:10825000AB619EE71E4B0293019B1E01029BF35AEA
:10826000002B2DD002998C19A068002828D0012A53
:1082700026D1FA889B189BB27352A189994217D3D1
:108280009B1AC018B96803F01FF9029BA289F35A20
:10829000934200D07DE700222B81A3882B80A36826
:1082A0006B60029BF2520B4A53680133536070E7D4
:1082B000084A9368013393600198FFF733FF68E73A
:1082C000044A536901335361F6E7C0462267FF1F32
:1082D000B867FF1F2867FF1F70B5051E15D10B4C2F
:1082E0000B4B1880230058331870606D002802D0A3
:1082F00003F03AF86565250050356068002801D024
:1083000003F032F80834AC42F7D170BD5C67FF1F50
:10831000AC67FF1FF0B51700A12285B09200019352
:108320004243394B06001B680C009B18D933FF33BE
:108330001D78FDF741FF0430854204DD3000FDF774
:108340003BFF0430C5B2BD4207D33A0000213000E4
:10835000019B03F069FA05B0F0BD2900380003F075
:108360007BF82300C6B250331E700393019B290093
:108370006365380003F0A8FACBB20293002B02D059
:10838000039B01361E7000262300503303931B7895
:10839000B34204D8606D002831D10020DBE7029A97
:1083A0002800002A04D0013B1000B34200D028006E
:1083B000F700E719387003F037F9786000280ED01D
:1083C0003A78019903F080F8019A3B780136D31886
:1083D0000E4A0193D369F6B20133D361D4E7039B0C
:1083E00018706065A74205D1084A1320D36A01338B
:1083F000D362B0E7606802F0B7FF0834F2E702F03A
:10840000B3FF00236365C8E73409FF1F2867FF1F18
:10841000F7B50D0007000421686803F0B5F92B8952
:10842000040003702B891B0A43702B8883702B88F0
:108430001B0AC3702E8902250436F6B2FB2E15D80E
:108440001B4B9F4214D10C2002F0F6FF1135011E88
:108450000CD0902303708E3B0371043B4380154B7B
:108460008460C680187803F097F800252800FEBDC8
:108470005C237B43104AD3180093583301931B7835
:10848000002B0FD10300320038000099FFF742FFA4
:10849000019B05001B78002BE8D13800009903F000
:1084A000FBF8E3E7054A0725536A01335362DDE72A
:1084B000FEFF00002067FF1F5C67FF1F2867FF1F8C
:1084C000F0B587B0009017200F0016000193FFF75A
:1084D000F2FD1325041E19D00C98031E02D0019939
:1084E000201D9847030AE370052302AAA0700430F8
:1084F000908127700098667003A993800494FFF719
:1085000087FF051E02D0200002F02EFF280007B0D2
:10851000F0BD0000F0B587B01F000CAB1B780391D5
:10852000059301210DAB06001C78049200F0D6F8EB
:108530001425002821D02000FFF77EFD0135041E00
:108540001BD01149059B0A7803700132D2B2131E69
:10855000C68001D101231A000B7022713000049BE8
:1085600003990097FFF7ACFF051E09D123002100F6
:108570000648074A093303F0EFF8280007B0F0BDBA
:10858000002363802370F8E72467FF1F0F8000112A
:1085900030750000F8B505000E00064C064F236844
:1085A000002B02D03100280098470434BC42F6D199
:1085B000F8BDC046C867FF1FDC67FF1F0123064ADE
:1085C0005B425380002313715362044A136053606B
:1085D0009360D36013617047DC67FF1FC867FF1F9C
:1085E0000200002310B506499C000859002801D15B
:1085F000625010BD0133052BF6D11320F9E7C046B8
:10860000C867FF1F034A5388181A43425841404223
:1086100010407047DC67FF1FF0B585B002930AABCE
:108620001F780CAB1B88009008000E00019203938A
:10863000FFF7E8FF05001120002D1BD10E48FFF7C2
:10864000E1FF04001520002C14D006220B99A7711D
:10865000E01D02F039FF019B30002371029B2900CD
:108660006371009B66802370039B6562E381FFF763
:1086700091FF280005B0F0BDFFFF000010B5FFF727
:10868000C1FF04000220002C12D060880121FFF7F6
:1086900081FF606A002801D003F086F828220021BB
:1086A000200002F0E9FE012300205B42638020717C
:1086B00010BD000030B5074A074C558801001378FB
:1086C0000020A54204D05B1A59424B415842104049
:1086D00030BDC046DC67FF1FFFFF0000084A10B531
:1086E00001230C00904208D0FFF78CFF031E04D03A
:1086F000037923405A1E9341DBB2180010BDC046D7
:10870000FEFF0000024B1879431E9841C0B270472B
:10871000DC67FF1F70B504000D001600FFF772FF45
:10872000002804D10D4B9C4200D0143070BD416A2A
:1087300003790520002907D012221A40102A02D1FD
:108740000520002EF2D10F20DB06EFD5897E0C200C
:10875000A9428941494249420840E7E7FEFF00003B
:10876000030010B5002800D110BD0348034A41881A
:108770009142F9D09847F7E7DC67FF1FFFFF000041
:10878000002330B5C45CCD5C6C40D4540133102B55
:10879000F8D130BD0F23002210B5C45C6400224321
:1087A000CA54C25CD209013BF7D210BD02000100DD
:1087B00010B52032103102F09FFF10BDF0B58BB024
:1087C0000390102005931700049102F0B5FE00906D
:1087D000102002F0B1FE009B13240190002B05D065
:1087E00000280CD11324009802F0DEFF019B002B1F
:1087F00002D0180002F0D8FF20000BB0F0BD10200E
:1088000002F09AFE0600102002F096FE13240500E6
:10881000002E00D1AEE0002819D01022002102F075
:108820002BFE32002900039802F066FF041E0ED1D1
:1088300033787F2B51D830000099FFF7ABFF009BB6
:108840001B787F2B53D801990098FFF7A3FF3000C6
:1088500002F0AAFF002D02D0280002F0A5FF002C94
:10886000C1D1102002F068FE0600102002F064FE64
:108870000290002E7CD0002878D03A000F322300DE
:108880000125121105D00F333B4015B25A42534116
:108890001BB26A1E1201002B33D0049BD2B298186F
:1088A0000099029AFFF76CFF013D10220021300071
:1088B00002F0E2FDADB2049F2D017D19AF4242D01E
:1088C000002C33D0300002F06FFF029B002B00D150
:1088D00089E7180002F068FF85E729003000FFF7FC
:1088E00059FF28002549009AFFF74AFFA7E729000A
:1088F0000098FFF74FFF28002049019AFFF740FF3B
:10890000A5E70F210F4004998A18D9B28F4208D9E0
:10891000D15C06A819540133102BF6D1029A0199A3
:10892000C0E7791A48424141C901F2E739003000F5
:1089300006AAFFF725FF3200039806A902F0DCFE25
:1089400010370400BAE7002CBCD13000029906AA07
:10895000FFF716FF320006A9039802F0CDFE0822A9
:1089600004003100059802F0AFFDABE71324A9E73E
:108970001324AAE7002800D06EE733E7F4BB001108
:10898000F0B58BB00F0016000225009000283FD0F4
:10899000002A3DD00B1DDBB21800029302F0CCFD83
:1089A0001135041E34D0FDF747FD05003A0000994B
:1089B000201D02F099FFEBB20393E3702B0CDBB2A6
:1089C0002F0A00936370FFB22B0E2370A7700193E0
:1089D000FDF72CFD1022010006A802F085FF210002
:1089E000029A04AB06A8FFF7E9FE051E0DD1039B12
:1089F00008223370009B04A9B370019B7770F37059
:108A0000301D02F071FFFDF71DFD200002F0CCFECD
:108A100028000BB0F0BDF0B58FB00D00149E039090
:108A200004920593002A03D1022420000FB0F0BD68
:108A3000002EF9D00398FFF7E5FD1424071EF4D0AB
:108A40007278337812021A43B3781B041343F27816
:108A500012061A43036A0192934201D30133E3D110
:108A6000002D03D03B7901249B07DED5082200218D
:108A700006A802F001FD059B13240433DBB21800A5
:108A8000029302F059FD051ECFD0059A04990430D7
:108A900002F02AFF04223100280002F025FF3900ED
:108AA000102210310AA802F01FFF2900029A06AB1B
:108AB0000AA8FFF783FE041E0FD1082206A908A802
:108AC00002F012FF0822311D08A802F02DFD012836
:108AD00007D101990398FDF7C9FC280002F064FE54
:108AE000A3E70124F9E7000070B51C4C05002368DA
:108AF000181E10D0002D14D11A78002A0CD1981C01
:108B0000083202F0E1FC02F01FFE0135002808D116
:108B100023681D70012070BD0A331800082202F07E
:108B2000D3FC2368002BF5D0122002F085FC061E32
:108B30000DD0C1232168037045700231102202302C
:108B400002F0C2FC23683100587802F025FD20684D
:108B500002F02AFE00232360DCE7C0460468FF1F02
:108B6000F8B504002020FDF755FB0D4EA700BB59BA
:108B70000500002B0DD000280BD0D878FF2809D194
:108B800008492A000C55F35907480333611802F0CD
:108B9000E3FDF8BD290002F02FFC0028F0D1F8E732
:108BA0002068FF1F0868FF1FB99D001170B5064DB2
:108BB00084006359002B05D0D87802F0CDFCFF2249
:108BC0006359DA7070BDC0462068FF1F70B506009B
:108BD0008CB00C00150000213022684602F04CFCDD
:108BE00031001022684602F07FFE1D202100032282
:108BF000684402F079FE6846FFF7D8FD2D21040095
:108C000003222800694402F06FFE20000CB070BD02
:108C1000F0B50700160097B001931CAB1D78302209
:108C20001EAB00910AA800211C7802F025FC10223E
:108C300039000AA802F058FE1022002102A802F012
:108C40001BFC0722310002A802F04EFE072202ABF5
:108C50009818631E9C41019902F046FE02AB9C737A
:108C60002B005A1E934102AAD3730021102206A89A
:108C700002F002FC06221D9907A802F035FE1A2018
:108C800002ABC01806221F9902F02EFE1022009996
:108C90000EA802F029FE102202AB0EA908781C785B
:108CA000013A6040D2B2087001330131002AF5D197
:108CB0000AA8FFF77BFD102212A904000EA802F0FB
:108CC00003FC102206AB0EA908781D78013A684013
:108CD000D2B2087001330131002AF5D10AA8FFF79A
:108CE00065FD044310222098E4B212A902F0FCFDB5
:108CF000200017B0F0BD70B50E0014008CB001005C
:108D0000102268461D0002F0EFFD3100082204A881
:108D100002F0EAFD2100082206A802F0E5FD6846FF
:108D2000FFF744FD04001022280008A902F0DCFD32
:108D300020000CB070BDF8B506000D0000243719F6
:108D4000AC4200D3F8BD02F08FFD030A3B70631CF8
:108D5000DBB201379D4203D90234F054E4B2EEE7AE
:108D60001C00EDE773B506000C000225002819D0A1
:108D7000002917D0032101A8FFF7DDFF6B469A7980
:108D80003F231A40013313436A463000937101A90F
:108D90002200FFF71BFF051E04D10322E01C01A9DE
:108DA00002F092FB280076BD03785807DA08C00F5E
:108DB000D20080009B0710439B0F1843C0B270473E
:108DC00007230B40C908C9000B430370704700001C
:108DD00070B50400FFF7EAFE134DA4006359002BA1
:108DE00021D0186A002801D002F0DEFC2B59986EC1
:108DF000002801D002F0D8FC2B59D86E002801D0F1
:108E000002F0D2FC2B59186F002801D002F0CCFCE4
:108E10002B59586F002801D002F0C6FC285902F0E7
:108E2000C3FC00232B5170BD2068FF1F0E4B800038
:108E3000C35870B50C00002B0FD09D68002D0CD0CE
:108E40002B78201D0B706B784B70A97CFFF7B8FF57
:108E50002B7E23726B69E36070BD1022002120001D
:108E600002F00AFBF8E7C0462068FF1F014B1860BC
:108E70007047C0461C68FF1F074A030080008258E5
:108E800010B5002A06D0D088984203D1012901D11B
:108E9000FFF79EFF10BDC0462068FF1FF0B5264EAD
:108EA00095B087000B93BB590500099112200A92D7
:108EB000002B31D0D888FFF7A5FB04001420002C2C
:108EC0002AD0280010A9FFF7B1FFBB591E781D6AF0
:108ED000002E23D00895FDF7EFFA07000020FDF7DC
:108EE000F1FA0790A379E61D069310AD0CA9089836
:108EF00000F0E2FA0EA9280000F0D7FA0B9B0A99BD
:108F00000493069B09980293079B0396019300978D
:108F10000EAB0CAAFFF77CFE15B0F0BDFDF7CCFA46
:108F200006903000FDF7CEFAE31DA779079310AB4A
:108F300006000893DAE7C0462068FF1F30B50C4CE6
:108F400085002A59030085B00120002A0ED01800A0
:108F50006946FFF76BFF2B591A78D888054B002A12
:108F600000D1054B6A46072100F0D9FB05B030BDA2
:108F70002068FF1FAB940011B994001130B5094C63
:108F80008500295985B010226846253102F09CFAE7
:108F90002A591121044BD0886A4600F0C0FB05B065
:108FA00030BDC0462068FF1F5595001130B5094CF3
:108FB0008500295985B010226846353102F084FABF
:108FC0002A591121044BD0886A4600F0A8FB05B04D
:108FD00030BDC0462068FF1F93950011F7B54D4F77
:108FE00086001020F4590D0002F0A6FAF359206211
:108FF000186A132200286CD0033A29009C6802F0FA
:1090000063FAF3591A780192002A58D11E6A227D18
:10901000317B944651400122019F114201D16746A4
:109020001740217D914339432175377B4F40BC4622
:1090300060460027800701D44F0817400121022015
:109040008F40227D82433A432275377B5740BC468E
:1090500060460027400701D497080F400420227D76
:10906000BF0082433A432275627D002794466046E2
:10907000727B42400A4201D167460F400121627D66
:109080008A433A436275777B5740BC466046002767
:10909000800701D457080F400220627D7F00824381
:1090A00017436775767B00227E40760701D4BA08A5
:1090B0000A400426617D9200B1430A4362756A78D2
:1090C000002A08D06278002A05D005220533DA7715
:1090D00000221000FEBD04222979114205D1A17C95
:1090E000114202D10533033AF1E7019A21782C7835
:1090F000002A02D10A002100140018220429E8D80D
:10910000042CE6D805206043034A05331218525C4C
:10911000DDE7C0462068FF1F04BC001110B50A003F
:109120001121024B00F0FBFA10BDC046EF95001173
:109130000B0030B587B001AD2B806B4604001100E9
:10914000981D082202F0C0F92A000B212000024BD2
:1091500000F0E5FA07B030BD1796001110B50A000F
:109160001121024B00F0DBFA10BDC0466B960011D6
:1091700013B50B0011006A4613706B4604000622FB
:10918000581C02F0A1F96A4608212000014B00F0AA
:10919000C6FA13BD8B96001110B50A001121024BBF
:1091A00000F0BDFA10BDC046DB9600117FB505008A
:1091B0000B4BAA00D4580800002C0FD0666F237FF9
:1091C000E28821780396266F0296E66E0196A46ED9
:1091D0000094FDF709FC2800FFF7FAFD7FBDC046AB
:1091E0002068FF1F10B51721FFF7E0FF10BD00003A
:1091F00070B50A000D00064B0221040000F08FFA42
:10920000060029782000FFF7D1FF300070BDC0466E
:10921000BB95001170B586B000236A461370836851
:1092200004001D78681E0A2859D801A902F024FB01
:10923000060633373B3F43474B4F5300180000F0BF
:1092400042F9062312284BD000281BD16088FFF773
:10925000D9F90823002813D04279002A47D1264B98
:109260001A78072312070BD5244B1A680723002A04
:1092700006D01668002E03D0290001AAB0470300CB
:109280006A4613706B461B786088002B2AD1FFF763
:1092900067FC06B070BD180000F06CF9D4E7180048
:1092A00000F087F9D0E7180000F093F9CCE7180038
:1092B00000F0ADF9C8E7180000F0C3F9C4E71800E2
:1092C00000F0F6F9C0E7180000F0F6F9BCE7180066
:1092D00000F013FAB8E7180000F013FAB4E7072318
:1092E0006A46137069466088FFF782FFD1E705235D
:1092F000012AC5D1024BB8E7AD66FF1F1868FF1FF2
:109300001C68FF1FF8B52C4F8600F35904000D00B0
:10931000002B40D0DA8882423DD15A78062A33D1D8
:109320001A78002A2ED0012099681A6A097D014214
:1093300006D0157B054203D007225A700120F8BDE4
:109340000220014204D0157B054201D00922F4E736
:109350000420014204D0127B024201D00B22ECE730
:10936000164B1B68002BE9D05B68002BE6D0200071
:109370009847BB5900215B78122BDFD12000FFF703
:1093800015FFDBE70E4BECE7112A04D1002900D0D2
:1093900032252900F2E7002D08D12000FFF732F92D
:1093A000002803D010230279134303712100280001
:1093B000FDF798FAC2E7C0462068FF1F1868FF1F34
:1093C0001C68FF1F70B50E4E8500AB590400002BC2
:1093D00013D01B78002B11D10A4B1B68002B04D033
:1093E0005B68002B01D02000984773595B78122BE3
:1093F00003D100212000FFF7D9FE70BD024BECE73E
:109400002068FF1F1C68FF1F1868FF1F094B8000A2
:10941000C3581020002B0CD01A6A002A09D09B6870
:10942000002B06D0127A1B7E101C9A4200D9181C01
:10943000C0B270472068FF1F70B503000D00140014
:109440000220002A30D000292ED013700B78081D7E
:1094500053704B789370FFF7A7FCE0700120022156
:109460002B7A23716B7B034063716A7B0A40134341
:10947000042263716E7B1640334363716E7BF60882
:10948000F600334363712B7B0340A371287B0140BB
:1094900000200B43A371297B0A401343A3712A7B4D
:1094A000D208D2001343A37170BD10B50A000100A9
:1094B0000120FFF7C1FF10BD10B50A000100022016
:1094C000FFF7BAFF10BD70B506000C000220002E99
:1094D00030D000292ED07378201D0B70B3784B70DC
:1094E000F178FFF76DFC01223579257271794B1007
:1094F0000800134093401040034388101040800040
:10950000C9080343C9000B436373B1794B100800CA
:109510001340934010400343881002409200C90852
:109520001343C9000B4321202373FCF773FE8542CC
:1095300001D2122070BD2220257AFCF76BFE8542F5
:10954000F7D823781820042BF4D86378012BF1D8AE
:109550000020EFE7030010B50220002909D0002BFE
:1095600007D00322481C0A7019000D3201F0ACFF2D
:10957000002010BD03000222080010B5002B06D009
:10958000002904D00E32591C01F09EFF0022100069
:1095900010BD030010B50220002909D0002B07D010
:1095A0000422481C0A7019000C3201F08DFF0020C3
:1095B00010BD10B5FFF7DEFF10BD0300022000292B
:1095C00006D0002B04D0052200200A701B784B70B7
:1095D000704703000220002B08D0002906D05B78DA
:1095E00000200B70013B082B00D918307047030096
:1095F00010B50220002909D0002B07D00622481CF4
:109600000A7019000A3201F05FFF002010BD10B58A
:10961000FFF7B0FF10BD02000B00022010B50029BB
:109620000ED0002A0CD007211970118859701188AA
:10963000090A997011180822D81C01F045FF002072
:1096400010BD03000A00022010B5002B0CD0002929
:109650000AD099785878090201431180901CD91CCE
:10966000082201F031FF002010BD030010B50220D8
:10967000002909D0002B07D00822481C0A701900C5
:10968000921801F021FF002010BD02000B00022003
:1096900010B500290BD0002A09D0092119701178C2
:1096A00018185970511C062201F00EFF002010BD41
:1096B00010B5FFF75FFF10BD02000B00022010B5D0
:1096C000002A09D0002907D05178197011180622F4
:1096D000581C01F0F9FE002010BD030010B5022057
:1096E000002909D0002B07D00A22481C0A70190053
:1096F000063201F0E9FE002010BD10B5FFF73AFF79
:1097000010BD02000B00022010B5002A06D000296F
:1097100004D018005178FFF753FB002010BDF0B5BE
:1097200085B017001E006A460623050008009181D7
:109730009380FEF7C0FC1324011E02900CD0380069
:10974000B047041E05D1280001A9FEF76FFA041ED8
:1097500002D0029801F008FE2800FFF701FA20006D
:1097600005B0F0BDF0B504008BB0019115000021EB
:10977000102202A801F080FE334EA700B85900283D
:109780003CD0C388A34239D10378002B36D142782C
:10979000062A18D102000100553235310C3006ABD3
:1097A000FFF7A9FA002829D12000FFF72FFE0200B9
:1097B00006A902A801F088FE200002A902F09CF888
:1097C00001200BB0F0BD816E002917D00B8A112A41
:1097D00028D19D420ED101981231093A01F0A4FE20
:1097E000012807D1BB5920009D6EFFF70FFE29000D
:1097F0000200DEE732212000FFF7D8FC2000FEF750
:1098000001FF061E1BD0416A002918D00B8AAB420B
:1098100015D108220198123101F086FE01280ED1DF
:10982000716A0AE09D42E9D108220198123101F0E3
:109830007BFE0128E2D1BB59996E8A7EB9E72000F0
:1098400002F082F8BCE7C0462068FF1FF0B56B4D00
:1098500087007E5985B0337802900393002B00D0A7
:1098600087E0B368346A01937078062817D1012223
:109870001B7D134202D0217B114218D102221342D8
:1098800002D0217B114251D10422134203D0237B09
:10989000134200D08BE0019B5A7DEB5991E00738D1
:1098A0000428F8D801F0E8FF032E42678300B36E66
:1098B000002B03D11C2001F03FFEB066EB599C6EDB
:1098C000002C1CD010220021200001F0D5FD0298B0
:1098D000FFF79CFD01002000FFF72DFA01F0C4FF07
:1098E0002082200008211230FFF725FA0298FFF7A6
:1098F0008DFDA076EB592100D888FFF70FFC0822D8
:10990000EB591CE0B36E002B05D01A00198AF088C1
:109910001232FFF70DFC0222019B197DEB59114217
:109920003DD0207B10423AD0073208E0F488FCF7A3
:10993000DBFD01002000FFF711FC0A22EB595A70F1
:10994000029B9C002A595378073B042B11D8D088DE
:10995000FEF758FE00284ED0C3895A08D21828496D
:10996000029B0298CB542B5941180433254801F02F
:10997000F3FE05B0F0BDFCF79FFD0300012083421C
:1099800001D100200393EB59DE88FCF79BFD03997E
:1099900002003000FFF7ECFB019AEB59117D042225
:1099A00011420CD0217B114209D00B22C7E7F68867
:1099B000FCF73CFD01003000FFF7EEFB6BE7019A7E
:1099C000527D01210A4204D0607B084201D00C2262
:1099D000B5E702210A4204D0607B084201D00E2282
:1099E000ADE704210A4204D0627B0A4201D0102272
:1099F000A5E71222A3E7FA225200B0E72068FF1F72
:109A00002468FF1FC39D001110B5064B1A7804236C
:109A1000100018401A4200D00348FFF727FA002030
:109A200010BDC046AD66FF1F3845FF1F70B504006E
:109A3000FFF7D4FA051E43D12000FFF77FFA234E2B
:109A4000A400A0598268937CDB0708D50321036A30
:109A50001B790B40012B02D1017F0B430377431D80
:109A6000D97F8B1E022B0DD8022900D00121C0887E
:109A7000FCF790FF042133591A7F59700A431A7773
:109A8000280070BD01290CD102231022437000214F
:109A90000C3001F0F1FC305910213530FFF74BF953
:109AA000EEE70529ECD10223D118437010220C30C7
:109AB00001F00AFD04233259117F0B431377EAE7C3
:109AC00008251828DCD1053DDAE7C0462068FF1FCD
:109AD000F0B58BB0059143887E4F9E00F459150078
:109AE0000493002C15D1012902D000200BB0F0BD49
:109AF000101D57781678FFF757F9EB68320002937C
:109B00002B7A0499019300903B002000FCF70CFF96
:109B1000EBE7E388049A934201D00820E6E7237834
:109B2000012B00D1D4E0059B581E092800D9CFE0B5
:109B300001F0A2FE05CE0A29CC506C859AB229000C
:109B40000498FFF773FFD1E7200029001022453069
:109B500001F0BAFCB9594B78042B02D1013B4B7090
:109B6000C3E70B000A00253335320C310498FFF7A8
:109B700095F90498FFF702FA0522431E9841BB5954
:109B8000C0005A70B2E7200029001022553001F0C1
:109B90009BFC049B4F4C9D00295904980A0006AB7E
:109BA00055320C31FFF77AF929591022453106A8B0
:109BB00001F0BAFC012808D10498FFF7F7F90590E5
:109BC000002804D106222B595A7005988EE70823E5
:109BD0000593FAE763780C2B7AD1E36E002B03D15F
:109BE0001C2001F0A9FCE066BB59D86E00286FD09C
:109BF0001022290001F068FCBB590498DC6EFFF7C5
:109C000005FC0D22A076BB595A706EE7E06E002865
:109C10005ED063780D2B5BD12B8808220382A91CB0
:109C2000123001F051FCBB599A68517D0222114259
:109C300026D0186A407B104222D00C32E4E76378C9
:109C40000E2B45D1236F002B03D1162001F074FC9D
:109C50002067BB59186F002803D01022290001F09B
:109C600033FC0F22BB59CFE763780F2B30D1206F25
:109C70000622691C103001F027FCBB599A68517DFF
:109C80000422114203D0196A497B1142D5D1002127
:109C90000498FFF78BFA28E7636F002B0DD0BB59B0
:109CA000586F0028F3D01022290001F00DFC01228A
:109CB000BB5952425B6F1A61E9E7142001F03CFC8A
:109CC000BB5960675B6F002BE9D126E72978DFE796
:109CD00007200BE72068FF1F10B5064C207001F02D
:109CE00013FB06212078FDF791FF0348FEF778FC6F
:109CF00010BDC0463368FF1F798E001100200BB2E3
:109D000070B50D00834216DA264B187801F00CFE70
:109D1000041E0DD00378922B0ED0A02B37D0224BEF
:109D20001878FF283AD0210001F036FC002835D100
:109D300080200002684070BD43780E2B0BD03E2B74
:109D4000EDD18378052B12D0082BE8D1817980885A
:109D5000FFF7D8FA08E0154B82889A42DFD1836872
:109D60001878591CFEF7C0FE002817D1D7E7104B12
:109D70001B785B0712D50F4B1B68002B0ED09B681E
:109D8000002B0BD0C289811D80889847ECE7FFF734
:109D900041FAA068002801D001F0E6FA200001F0A5
:109DA000CBFCC5E73368FF1F3145FF1F18200000BB
:109DB000AD66FF1F1C68FF1F10B50078FFF712FA91
:109DC00010BD10B50078FFF7FDFA10BD0C2343431A
:109DD000084A10B59B185A68002A03D0012901D1FE
:109DE000904710BD9B68002BFBD00029F9D1984704
:109DF000F7E7C0465068FF1F01238340094A10B5AA
:109E0000946B1C439463506B98435063D46B200055
:109E10009843012901D120001843D063116B0B43F3
:109E2000136310BD00800040F0B500240127154BDE
:109E300085B0DA6B144E03921A6C0192DA64019BBE
:109E4000E3403B4217D0039DE5403D400295E5B21B
:109E500002992800FFF7BAFF316A736A002908D017
:109E60003900002B01D0029979402800FFF7C4FF88
:109E700001E0002BF9D101340C36172CDFD105B0ED
:109E8000F0BDC046008000403468FF1F064B012132
:109E90005A68C2400A4204D01B68C34018000840F8
:109EA00070471B6DF9E7C046008000400122064B59
:109EB0008240002903D0D9680A43DA607047D96824
:109EC0009143D960FAE7C0460038004030B503241A
:109ED00044430F4BE25C1B199C785D7801232D1BDA
:109EE0000135AB40013BA340A140DB430C001228ED
:109EF00007D808499200521811681940214311608F
:109F000030BD054A11680B4023431360F8E7C04693
:109F10004BBC001108F0004014F00040C21F70B5A7
:109F2000D4B20623092C0BD80125084C95400029F2
:109F300008D00021FFF7CAFF23682B4323600023CA
:109F4000180070BD2368AB43F8E7C04600380040F6
:109F5000214BF0B51B185B78022B21D1032444431D
:109F60001E4A1F4EA35C12199478012215008540E9
:109F7000B76B013CE4B23D43A240B563194C1228D3
:109F800015D89B0000290CD117495B1899680A4322
:109F90009A600123205C154A834011680B431360CB
:109FA000F0BD11495B18996891439960F1E70E4B38
:109FB00000290DD159690A435A61225C1328E8D05F
:109FC0000123203A93400A49086803430B60E7E7FE
:109FD000596991435961F0E73468FF1F4BBC001188
:109FE0000080004090BC001100F00040A0F0004054
:109FF000A4F00040F8B500241B4E1C4D1C4B1B5D0B
:10A00000012B1FD1194A9269E2401A420BD001225A
:10A01000B25693402200143AD2B2022A09D8154906
:10A020004A6913434B61013402360C35172CE5D1D4
:10A03000F8BD0022B2560F499200521891680B43A6
:10A040009360F0E7022BEED1E7B23800FFF71EFF76
:10A0500001235840C1B23800FFF77AFF3800FFF7FC
:10A0600015FF6877DFE7C0461DBC00113468FF1F8D
:10A070003568FF1F00F00040012202388240054B86
:10A08000002903D059690A435A61704759699143BD
:10A090005961FAE700380040F8B50E0001210F00C1
:10A0A0008740114A0400D368FD43BB43D360831E3D
:10A0B0008B4201D8FFF7E0FF00212000FFF72EFFC1
:10A0C0000A4A0B4B5168012E05D139431B195160C7
:10A0D0005E700020F8BD2940516002221C19627098
:10A0E0009A6915409D61F4E7003800400080004007
:10A0F0003468FF1F012210B58240074B002906D0AB
:10A1000019680A431A600121FFF7C6FF10BD1968DC
:10A1100091431960F7E7C046008000400C2370B5FA
:10A12000002543430A4A29009B181D70094B04006F
:10A130001B185D70FFF7B0FF0123A34006492800FC
:10A140000A681A430A6005490A689A430A6070BDA2
:10A150005068FF1F3468FF1F34800040308000408B
:10A1600070B504000E00FF2813D003250540FFF74B
:10A17000D5FF084AA3089B009B183F22ED00AA4088
:10A18000AE40196820009143314319600121FFF767
:10A190008DFE70BD18380040F8B50C244443134BB5
:10A1A0000500E4186368002B03D1A3681220002B7C
:10A1B0001AD0022201270E4B00215B195A70280089
:10A1C0002770FFF769FF63681E1E08D0A3683E0072
:10A1D000002B04D02800FFF759FE4640F6B22800B5
:10A1E0003100FFF709FE0020F8BDC0465068FF1F90
:10A1F0003468FF1FF7B5C420FF222B4B800019588D
:10A20000002491433F3A0A431A508022274F5202BA
:10A21000274E1A60274B1D5D002D21D0A31E012B58
:10A2200003D80121E0B2FFF727FF012D18D11F4B02
:10A230009B69E3402B4213D0E3B218000193FFF770
:10A2400025FE01000198FFF755FFE3B2143B022BF6
:10A250001DD801217156184A8D405369AB43536193
:10A260003B7F002B0DD0E5B22800FFF795FF2800BB
:10A27000FFF70CFE7B7F0100834202D02800FFF72E
:10A28000A5FD01340C370236172CC3D1F7BD0121CF
:10A2900000237156F3568D40074A9B009B189A681D
:10A2A000AA439A60DCE7C04600E100E03468FF1F83
:10A2B0001DBC00113568FF1F00F0004010B50121E2
:10A2C0000400FFF7E9FE0123044A002011194B7036
:10A2D000A34091690B43936110BDC0463468FF1FD2
:10A2E00070B50E0015000400FFF718FF0C23634340
:10A2F000094A20009B189D605E60FFF74DFFF0212A
:10A30000064B074A8900051E5A5002D02000FFF76D
:10A3100005FF280070BDC0465068FF1F0000FF1FEA
:10A32000299E001170B5134D07202C78002C1FD1E9
:10A33000982221005200280001F066FA0123C4206F
:10A34000FF222B700C4B80001C635C630B4B1C606A
:10A350005C600B4B195891433F3A0A431A508022D4
:10A3600052021A600D20074A074901F0A5FA2000A1
:10A3700070BDC0463468FF1F00800040A0F0004060
:10A3800000E100E0F5A10011F59F0011030010B5F8
:10A390000620072B09D8054A137000F0EDFFD721DE
:10A3A0000020034B034A89005A5010BD6045FF1F2F
:10A3B0000000FF1F151BFF1F70B51D0002240C2994
:10A3C00010D8094ACA40D2070CD5FBF72FFF041E4C
:10A3D00008D1059A04992800FBF744FFFCF7B2FD69
:10A3E000FFF712FB200070BD1210000030B50D7891
:10A3F00002232C009C43184201D02B431C0008254B
:10A400002300AB43284201D02B00234320241D000E
:10A41000A543204201D01C4325002A230D70184279
:10A4200004D011781E3B0B43137030BD0028FCD1C3
:10A430000C2113788B43F7E7F8B51D0006AB1B889A
:10A44000140007AA0E000B201778002B27D10A78DA
:10A45000022A49D14A68507811780002244A0843F8
:10A460008018042840D801F007FA03121D1B2300AE
:10A47000F06801F0B9F9021CC0B2B84200D93A1C28
:10A48000D2B22000F1682A8001F01EF806E0022214
:10A49000F3681B882A8023701B0A63700020F8BDB4
:10A4A0000622EEE701232B80F3681B782370F5E783
:10A4B000F368002B16D008222A801A8822701A8886
:10A4C000120A62705A88A2705A88120AE2709A8838
:10A4D00022719A88120A6271DA88A271DB881B0ADB
:10A4E000E371DBE72B80D9E701202B80D7E7C0465B
:10A4F00000D6FFFFF7B516000A781D0008AB1F88CD
:10A500000C000123022A18D14A6850781178000201
:10A510002B4A0843801803280FD801F0ADF9022513
:10A520004439E06801F060F9C0B20723B84204D3AF
:10A530007B190193152B02DD0D231800FEBDE06889
:10A540002A003100C01900F0BFFF6B4600209B8835
:10A55000E268D0541B4B1B68834203D01B688342C4
:10A5600000D098470023E8E70B23002FE5D1022D08
:10A57000E2D1737832781B021343E2681380114BE7
:10A580001B68002BEED01B68002BEBD00120E8E706
:10A590000B23002FD1D1062DCED12A003100E06847
:10A5A00000F092FFDEE70B23002FC6D1012DC3D1AF
:10A5B00032787533012AC0D8E3681A70D2E7C046F2
:10A5C00000D6FFFF406AFF1F70B50C00150007287A
:10A5D00037D801F051F9041436361B36242E1820D2
:10A5E00015290BD8184E16220021300000F044FF28
:10A5F00022002900300000F067FF002070BD182005
:10A600000229FBD11288114B1A80F6E7182008297D
:10A61000F4D10A000E48290000F0C6FEEDE718202C
:10A620000129EBD10B4B10780B49DA69FFF7DEFEFD
:10A63000E3E718200129E1D1064B10780749DA6BCE
:10A64000F4E70220DAE7C046286AFF1FDE45FF1F55
:10A65000D445FF1F6445FF1F8C45FF1FAC45FF1FFE
:10A66000030010B50020DB0704D50721024A034888
:10A6700000F08CF810BDC046A8BC00116445FF1F57
:10A68000054A03001068002803D082889A4201D14D
:10A69000806870470068F6E7446CFF1F0A88030073
:10A6A00008009A4204D08A8804309A4200D00020E0
:10A6B00070470000F8B5F82200230D4F0D4E796861
:10A6C000050042433370994200D07B600A4C002160
:10A6D000200000F0D1FE00231A007C60AB4202D1C2
:10A6E00000203370F8BD01332280DBB2F834F5E787
:10A6F000446DFF1F406DFF1F486CFF1F73B56B4615
:10A7000001900600684615001980FCF74DFF041EF5
:10A7100011D1002D0FD07689002E11D00C2000F021
:10A720000BFF00280ED0084A0460136886808560FD
:10A73000002B02D11060200076BD1A001B68F7E7DD
:10A740000224F8E71324F6E7446CFF1F01210022DE
:10A750000A4B10B549420A4C198099809A719A7037
:10A76000084B2070012019805A60FFF7A3FF207862
:10A77000FCF778FF0448FDF733FF10BD486AFF1F60
:10A780004C6DFF1F446DFF1F39A80011022310B547
:10A79000002802D0FFF7B2FF0300180010BD000030
:10A7A000030010B50020DB0704D50421024A03484A
:10A7B000FFF7A4FF10BDC046BCBC0011E445FF1F5D
:10A7C000F0B50E2687B003930CAB1F8802ABF618CA
:10A7D0000500080031000292FDF768F8040001202E
:10A7E000002C0FD03088FFF74BFF03000E20002B0A
:10A7F00008D05E68002E05D021002800039B029A35
:10A800000097B04707B0F0BD0A4B10B5984207D18A
:10A810000122002352420A808B708A808B7110BD06
:10A82000FFF73CFF0028FAD001235B42038000239E
:10A830008370F4E7FFFF0000F8B5050001290AD195
:10A84000134E00243388F827AB4219D02800114951
:10A85000FFF7DAFF06E0022904D10139FDF73EFFD8
:10A860000028EDD0F8BD3B0063437268D018D35A7E
:10A87000002B09D03A00002100F0FEFD0134E4B2C3
:10A88000054B1B78A342EED801235B423380DDE702
:10A89000446DFF1F486AFF1F406DFF1F10B5FFF793
:10A8A000FDFE03000020834200D0987810BD000018
:10A8B000F0B589B01C000EAB80CB03901E8810ABA6
:10A8C0001B78049202930B7A0D00DB0616D42B78CA
:10A8D0000593022B24D00498FFF7D2FE002812D053
:10A8E00003689C46002B0ED0029B22000193290096
:10A8F0003B00644603980096A04705E00498FFF7E4
:10A90000BFFE002802D10E2009B0F0BD8368002BE5
:10A91000F9D00A222900039898470028D7D0F3E7F6
:10A920006B6858781A786B4B000210439842D2D863
:10A93000043B984210D2684B984242D015D8674BDE
:10A94000C0180128C7D80B20002EDDD1EB681A787B
:10A9500059683A80200028E0614BC018032800D9CC
:10A9600079E000F089FF846A789E5E4B9842B2D10C
:10A970000B20002EC8D101233B80EB6831001B78EF
:10A9800023706889013080B2FCF790FF3A88031E7B
:10A990000ED0017802328A183A8042896270428968
:10A9A000120AA27059680278E01C00F08DFD06E0E2
:10A9B00004323A8031000422601C00F05DFD00206A
:10A9C000A2E70B20002E9FD1EB6807A91E88042365
:10A9D0003B80330A300026706370FCF767FF051E6A
:10A9E00028D004AB9A890E2304A95B183E49C66897
:10A9F000FCF7D0FF00280BD12B783C486A680599FA
:10AA0000FBF786FB002803D1012304AA5B42D38114
:10AA10003278022A06D17168201D00F055FD3B886E
:10AA200002333B800E2304AA9B181B88A3701B0AC9
:10AA3000E370C4E704ABDE81F4E70B20002E00D006
:10AA400062E7E9680398FFF729FF02233B80207043
:10AA5000000A6070B3E70B20002E00D054E70222FA
:10AA6000EB681B883A8023701B0A6370A7E7E868CD
:10AA700000F0BAFEC2B203000720B24200D243E7A0
:10AA80000DD00299DBB27118994202DB921BD3B24E
:10AA90000293029BE9681A003B8089195AE7002358
:10AAA000F6E70B20002E00D02EE70722EB683A8055
:10AAB0001A7822705A7862705A88A2705A88120ADC
:10AAC000E2701A792271DA886271DB881B0AA3713D
:10AAD00075E7C046042900000228000000D8FFFFE7
:10AAE000FFD6FFFF03280000FFFF0000ECBB0011B2
:10AAF000F0B58DB06B460020089120229B5E83420A
:10AB00003DDAA64B187800F00FFF071E32D003780D
:10AB1000B02B2CD10079023816281FD800F054FD34
:10AB200017001E001E001E0031001E0096001E00B1
:10AB30001D011E0052011E0073011E00CD011E00EA
:10AB400050021E001E001E008E021E00E302944BE7
:10AB500094491B8878880B80FBF71AF83800FCF7BB
:10AB60009BFF914B1B68002B01D0380098473800A1
:10AB700000F0E2FD8020089B0002434018000DB069
:10AB8000F0BDF6220021874800F076FC0BAA3B7B43
:10AB90007989388900923A000D32FCF79FFD040054
:10ABA000804B1B78002C3FD146E0804B7888059382
:10ABB0007F4B4100CB5A0BAE073BDBB2328802938E
:10ABC000002301937B4B210006930093059BFFF725
:10ABD0006FFE744D002810D1069B3A8A1B889A425A
:10ABE0000BD138000599123000F09EFC002804D0EB
:10ABF0002B7862899B00EB185A80162306A81B1835
:10AC0000328820007989FCF7C5FE2B7804009A0071
:10AC1000AA1851880029C3D00133DBB22B70002859
:10AC200007D006A9C98A9180634A12889A42BCD883
:10AC300002E0012149429180002B04D059497888D3
:10AC4000FAF7DAFF8AE73E890A2479E000253E898F
:10AC5000574B06937B88069A5B009B5A033B9D42A9
:10AC600002DB002DF0D05BE0162206A812183B7B19
:10AC7000798900923A0030000D32FCF72FFD0590E3
:10AC8000002858D04689017A7888FCF7F1FC041E28
:10AC900044D1464B78880793069B4100C95A454BDF
:10ACA0000439C9B206AAD28A06930291019400938C
:10ACB0000599079BFFF7FCFD041E2FD1069B394920
:10ACC0001A88931C002D26D14B807988384B490077
:10ACD000CB5A5119033B8B4220DD059B31485B89E0
:10ACE00041190B71A91C0135C9B2EDB20591451985
:10ACF0001B0A2B71059B2D490433181800F0E4FB47
:10AD00002C4B059A1B88D318DDB22C4B9E4205D0E4
:10AD10000136B6B29CE749889942D6D0002D0CD0B6
:10AD2000204C2800618800F0D7FB20702100788833
:10AD3000FAF772FF12E7059CF0E7002C00D183E7D9
:10AD40007B78142B00D109E716493B794E800B70B4
:10AD50000C717888FAF712FF00E7162406ABE418A6
:10AD600021003889FCF7A2FD011E00D1B7E17888E7
:10AD700022880F4C45002C5B0A4D013CE4B2029442
:10AD800000240F4B01940095FFF792FD041E00D0A4
:10AD900014E129007888FAF74FFFDFE64C6DFF1FBA
:10ADA000D044FF1F506AFF1F446AFF1F4A6BFF1FFA
:10ADB0008066FF1F406CFF1FCE44FF1FFFFF000097
:10ADC000526AFF1F162406ABE41821003889FCF7ED
:10ADD0006DFD011E00D182E178882288AE4C4500CD
:10ADE0002C5BAE4D013CE4B202947C89AC4B0194E7
:10ADF0000095FFF75DFD041E00D0DFE02900788894
:10AE0000FAF724FFAAE60025A44B1D803B00FE3381
:10AE10001B78A24A78880792AB4208D99E4B1288C9
:10AE20000693069943005B5A013B9A4203DB07995C
:10AE3000FAF716FF92E616246B00FB18059306AB93
:10AE4000E418059B21001889FCF730FD011E03D191
:10AE5000059B01241E8973E77888924B2288069C03
:10AE6000099343001B5B904E013BDBB2029300232E
:10AE700000960193099BFFF71BFD041E02D0059B62
:10AE80001E895DE77B88069A5B009B5A079A1088AB
:10AE900032881218934202DC1B1A013B33807F4C2C
:10AEA000023032880999001900F00EFB238832889D
:10AEB00001359B182380EDB2A8E70BAA3B7B79896B
:10AEC000388900923A000D32FCF708FC0025059005
:10AED000059B002B04D10A24002D00D16EE060E018
:10AEE000059B7888197AFCF7C3FB0100041E63D127
:10AEF000694C6C4B788806940993069B4400E45A8D
:10AF0000694B063CE4B20BAE328807930294019180
:10AF100000930599099BFFF7CBFC041E4CD1079BBE
:10AF20005E491B881A1D002D30D14A80059B5B4C61
:10AF30005A8963191A716B1C9BB2E318120A1A71B1
:10AF4000162306A832881B1879890598FCF722FD7C
:10AF5000FF21AA1C2E1D03350B00059092B2B6B23C
:10AF6000ADB2002803D006ABDB8AD9B21B0AA21807
:10AF7000651911712B714C4D301D2A8849492018D3
:10AF800000F0A2FA2B88F618B5B2A1E749889142E1
:10AF900007D17A8806995200525AEB18053A9A421C
:10AFA000C4DC3E4C2800618800F056FA2070210075
:10AFB0007888FAF75FFED1E5002DF2D13E89BFE631
:10AFC000162606ABF61831003889FCF76FFC3D00F9
:10AFD0000400FF3500282DD0037A9B060CD40022F4
:10AFE0007B893989788800923A000C32FFF7E8FBB8
:10AFF000041E10D03E8915E03088FFF741FB002881
:10B000001AD08368002B17D0210012227888984725
:10B01000041EE4D0EEE7AB78002B02D17888FAF773
:10B0200039FE0026AB78002B00D097E5002C00D12C
:10B0300094E585E60124DDE70E24DBE7162506AB63
:10B04000ED1829003889FCF731FC041E47D0037A3B
:10B050009B0611D4154A7B881188994203D0144865
:10B06000814207D11380134BF8261D780023D9B2F3
:10B07000A94221D30924A1E72888FFF701FB002872
:10B080002FD08368002B2CD021001222788898477B
:10B09000041EDFD092E7C0468066FF1F506AFF1F84
:10B0A000526AFF1F4A6BFF1F406CFF1F446DFF1F5A
:10B0B000FFFF0000406DFF1F31005943546801330A
:10B0C0006018615A0029D2D13C0008342100F822CE
:10B0D00000F0FAF921007888FAF7E4FD3EE5012452
:10B0E0006CE70E246AE71D4B1A887B889A4231D0A0
:10B0F0007888FAF7E1FD31E5F82305985168434374
:10B10000CD18C95A00291FD03B7A012B0BD16C886E
:10B11000AB887888AA1D0094FFF752FB041E02D06A
:10B1200000233B722E88F8220021280000F0A4F9A9
:10B1300000232B80059B0133DBB20593084B059957
:10B140001B78064A8B42D7D801235B421380002C20
:10B15000CED0F5E5002634000596EFE7446DFF1FDD
:10B16000406DFF1F70B504000E001500FFF796FA42
:10B17000031E08D131000548FFF790FA03001120A3
:10B18000002B02D01C8000209D7070BDFFFF0000CE
:10B19000F8B50B4F06003B780D001400FF2B0ED0C6
:10B1A0000A2000F049F9011E09D0B12303800023D1
:10B1B00046800371C5800481387800F0EDF9F8BD50
:10B1C0002546FF1FF7B50F0008A90600088809A942
:10B1D0000B240988002821D10234022B1ED1557876
:10B1E00013782D021D432B008B4301937334002BE6
:10B1F00014D1FB68300019000093FFF74FFB019C4E
:10B2000085420BD02A0030000099FFF7ABFF041EE7
:10B2100004D12A0030007989FFF7BAFF2000FEBD73
:10B22000F0B50E7885B003900AA805880120022E9B
:10B230000DD14C682778647824023C43054FBC420A
:10B2400005D10398DBB201960095FFF7BBFF05B06F
:10B25000F0BDC0460229000010B504000C4800F003
:10B2600083FA0C48A16B00F07FFA0B48E16B00F009
:10B270007BFA0A48216C00F077FA094B09481968F3
:10B2800000F072FA084B1B68002B00D09847FEE7CD
:10B29000BEBA0011D4BA0011E3BA0011F2BA00111B
:10B2A00004ED00E001BB0011506DFF1F002307B546
:10B2B00001A80193FFF7D0FF044A0548002110B50B
:10B2C000121A00F0D9F8F8F775FBFEE7546DFF1F6E
:10B2D0002846FF1F0000000001B40248844601BC5C
:10B2E000604700BF5D17000001B40248844601BCFE
:10B2F000604700BF9DA9000001B40248844601BC1C
:10B30000604700BFB352010001B40248844601BC4B
:10B31000604700BFC926000001B40248844601BC52
:10B32000604700BF053AFF1F01B40248844601BCD4
:10B33000604700BF5125000001B40248844601BCAB
:10B34000604700BF4D1F000001B40248844601BCA5
:10B35000604700BFB14E000001B40248844601BC02
:10B36000604700BFC9A9000001B40248844601BC7F
:10B37000604700BFD949010001B40248844601BCBE
:10B38000604700BF151BFF1F01B40248844601BC83
:10B39000604700BFB134FF1F01B40248844601BCBE
:10B3A000604700BFADAE000001B40248844601BC56
:10B3B000604700BF810E000001B40248844601BC12
:10B3C000604700BF3555000001B40248844601BC07
:10B3D000604700BF456B010001B40248844601BCD0
:10B3E000604700BF5952010001B40248844601BCC5
:10B3F000604700BF9538FF1F01B40248844601BC76
:10B40000604700BF5147010001B40248844601BCB7
:10B41000604700BF4939FF1F01B40248844601BCA0
:10B42000604700BF8552010001B40248844601BC58
:10B43000604700BFC56D010001B40248844601BCED
:10B44000604700BF1D4D010001B40248844601BCA5
:10B45000604700BF3D18000001B40248844601BCAB
:10B46000604700BF090E000001B40248844601BCD9
:10B47000604700BF5135FF1F01B40248844601BC3C
:10B48000604700BF154D010001B40248844601BC6D
:10B49000604700BF056A000001B40248844601BC51
:10B4A000604700BF913AFF1F01B40248844601BCC7
:10B4B000604700BF691F000001B40248844601BC18
:10B4C000604700BFC94A010001B40248844601BC7C
:10B4D000604700BFE94C010001B40248844601BC4A
:10B4E000604700BF350E000001B40248844601BC2D
:10B4F000604700BF0189000001B40248844601BCD6
:10B50000604700BF156B010001B40248844601BCCE
:10B51000604700BF4550000001B40248844601BCAA
:10B52000604700BFC537FF1F01B40248844601BC15
:10B53000604700BFCD4C010001B40248844601BC05
:10B54000604700BF3D4B010001B40248844601BC86
:10B55000604700BFF94C010001B40248844601BCB9
:10B56000604700BF1147010001B40248844601BC96
:10B57000604700BF3D3BFF1F01B40248844601BC49
:10B58000604700BF4136FF1F01B40248844601BC3A
:10B59000604700BFD13AFF1F01B40248844601BC96
:10B5A000604700BF594F010001B40248844601BC06
:10B5B000604700BFF30E000001B40248844601BC9E
:10B5C000604700BFB54C010001B40248844601BC8D
:10B5D000604700BF093DFF1F01B40248844601BC1B
:10B5E000604700BFD1A5000001B40248844601BCF9
:10B5F000604700BF055E000001B40248844601BCFC
:10B60000604700BF5522000001B40248844601BCD7
:10B61000604700BF6571010001B40248844601BC67
:10B62000604700BFB93BFF1F01B40248844601BC1C
:10B63000604700BF017F000001B40248844601BC9E
:10B64000604700BFA137FF1F01B40248844601BC18
:10B65000604700BFE530FF1F01B40248844601BCCB
:10B66000604700BFDD66010001B40248844601BCAA
:10B67000604700BFA54F010001B40248844601BCE9
:10B68000604700BF1D4B010001B40248844601BC65
:10B69000604700BF8932FF1F01B40248844601BCE5
:10B6A000604700BF7D18FF1F01B40248844601BCFB
:10B6B000604700BF2146010001B40248844601BC36
:10B6C000604700BFE928000001B40248844601BC7D
:10B6D000604700BF2526000001B40248844601BC33
:10B6E000604700BF2124000001B40248844601BC29
:10B6F000604700BF6DBC000001B40248844601BC35
:10B70000604700BFE548000001B40248844601BC20
:10B71000604700BFEDA5000001B40248844601BCAB
:10B72000604700BF8D12000001B40248844601BC8E
:10B73000604700BFC95C010001B40248844601BCF7
:10B74000604700BF434D010001B40248844601BC7C
:10B75000604700BFD91B000001B40248844601BC09
:10B76000604700BFA946010001B40248844601BCFD
:10B77000604700BFE53A010001B40248844601BCBD
:10B78000604700BFF134FF1F01B40248844601BC8A
:10B79000604700BF5549010001B40248844601BC1E
:10B7A000604700BFE13CFF1F01B40248844601BC72
:10B7B000604700BF014C010001B40248844601BC4F
:10B7C000604700BF75A9000001B40248844601BC6F
:10B7D000604700BF9930FF1F01B40248844601BC96
:10B7E000604700BF513AFF1F01B40248844601BCC4
:10B7F000604700BFDD52010001B40248844601BC2D
:10B80000604700BF291C000001B40248844601BC07
:10B81000604700BFB70E000001B40248844601BC77
:10B82000604700BFC51D000001B40248844601BC4A
:10B83000604700BF5118FF1F01B40248844601BC95
:10B84000604700BFE53BFF1F01B40248844601BCCE
:10B85000604700BF7132FF1F01B40248844601BC3B
:10B86000604700BFC521000001B40248844601BC06
:10B87000604700BF2951010001B40248844601BC61
:10B88000604700BFF53CFF1F01B40248844601BC7D
:10B89000604700BF0124000001B40248844601BC97
:10B8A000604700BF0D52010001B40248844601BC4C
:10B8B000604700BFC53F000001B40248844601BC98
:10B8C000604700BF1133FF1F01B40248844601BC2A
:10B8D000604700BF090E000001B40248844601BC65
:10B8E000604700BF193AFF1F01B40248844601BCFB
:10B8F000604700BF4551010001B40248844601BCC5
:10B90000604700BF311B000001B40248844601BCFF
:10B91000604700BFED4A010001B40248844601BC03
:10B92000604700BFC932FF1F01B40248844601BC12
:10B93000604700BFF54E010001B40248844601BCD7
:10B94000604700BF851F000001B40248844601BC67
:10B95000604700BF091B000001B40248844601BCD7
:10B96000604700BFE117000001B40248844601BCF3
:10B97000604700BF8B52010001B40248844601BCFD
:08B98000604700BF79180000C8
:10B988000003010302000303040205020602070084
:10B99800080309030A030B030C000D000E030F0331
:10B9A8001003110013031403150316037D3D001142
:10B9B800B13D00110000000002000000CAB90011EA
:10B9C800192A0F180A000000F1590000FD24000090
:10B9D80041460100E97C0011FD9C001151710011E4
:10B9E800ED7A0011F9520011F1AA0011714F0011FE
:10B9F800753F0011A5400011000000001616000058
:10BA08000200000014BA0011F4FFF3FFD2FC00009A
:10BA1800E541001100000000000000005475796144
:10BA28000042312E32003030303100676974687559
:10BA3800622E636F6D2F707676780054484232001C
:10BA4800020000005CBA0011292A282A272A262A7F
:10BA5800252A242A0A180000E204000071020000C6
:10BA680078EC0000744000001027000060F000002F
:10BA780006640000204E00000000000001000000E5
:10BA88001F501D00023CB40000011300120000000A
:10BA9800810200003031323334353637383941428B
:10BAA80043444546005048592B36325858504C5557
:10BAB8005330353034005B48617264206661756CC0
:10BAC800742068616E646C65725D0A004C522020B7
:10BAD800203D203078253038780A00504320202037
:10BAE8003D203078253038780A0050535220203DC8
:10BAF800203078253038780A0049435352203D20B9
:10BB08003078253038780A00FD5600115157001159
:10BB1800000000000200000028BB00116F2A6E2AF6
:10BB28001A18000001A00000000000006410B71DF2
:10BB3800C8206E3BAC30D9269041DC76F4516B6B53
:10BB48005861B24D3C7105502083B8ED44930FF015
:10BB5800E8A3D6D68CB361CBB0C2649BD4D2D386CB
:10BB680078E20AA01CF2BDBDFB349B5F8000008018
:10BB78000010000000000000535D0011DD7300118B
:10BB8800775D0011E5770011FB5D0011BB770011AF
:10BB9800715E001191770011C35E0011597900118F
:10BBA8002B5F0011597900115D5F001113790011A5
:10BBB800715E001149770011E95E0011F1780011FA
:10BBC8000000000000000000CF5F0011F1780011B4
:10BBD80031600011F5730011052A042A012A002A90
:10BBE8000229032801280028011800180000000075
:10BBF80000000000000000000000008701010201B1
:10BC08000201010201020303040103010101010110
:10BC18000303020103000D000E00100011001300C1
:10BC28001401070108010A010B011C011D0204028D
:10BC380005020702080219021A021C021D03010369
:10BC4800020317000201000504000807000B0A00A0
:10BC58001716001D1C010201010504010E0D01113A
:10BC680010011413011716011A19020201020B0A16
:10BC7800020E0D0211100214130217160305040315
:10BC88000807030B0A030E0D0001020307090A0B3C
:10BC98000E0F101112141718191A1B1F2021220039
:10BCA80039A40011F5A400110000000002000000F2
:10BCB800F2BB00110000000021B2001100000000DA
:08BCC80002000000F0BB0011B6
:020000041FFFDC
:1000000000000000D93E0011D0B90011CCB9001198
:100010003463FF1F0000000000000000000000002B
:1000200000000000000000000000000000000000D0
:1000300000000000000000000000000000000000C0
:1000400000000000000000000000000000000000B0
:1000500000000000000000000000000000000000A0
:100060000000000000000000000000000000000090
:100070000000000000000000000000000000000080
:100080000000000000000000000000000000000070
:100090000000000000000000000000000000000060
:1000A0000000000000000000000000000000000050
:1000B0000000000000000000000000000000000040
:1000C0000000000000000000000000000000000030
:1000D0000000000000000000000000000000000020
:1000E0000000000000000000000000000000000010
:1000F0000000000000000000000000000000000000
:1001000000000000000000000000000000000000EF
:1001100000000000000000000000000000000000DF
:1001200000000000000000000000000000000000CF
:1001300000000000000000000000000000000000BF
:1001400000000000000000000000000000000000AF
:10015000000000000000000000000000000000009F
:10016000000000000000000000000000000000008F
:10017000000000000000000000000000000000007F
:10018000000000000000000000000000000000006F
:100190001535FF1F5D33FF1FC16601000000000021
:1001A000000000000000000000000000000000004F
:1001B000000000000000000000000000000000003F
:1001C000000000000000000000000000000000002F
:1001D000000000000000000000000000000000001F
:1001E000000000000000000000000000000000000F
:1001F00000000000000000000000000000000000FF
:1002000000000000000000000000000000000000EE
:1002100000000000000000000000000000000000DE
:1002200000000000000000000000000000000000CE
:1002300000000000000000000000000000000000BE
:1002400000000000000000000000000000000000AE
:10025000000000000000000000000000000000009E
:10026000000000000000000000000000000000008E
:10027000000000000000000000000000000000007E
:10028000000000000000000000000000000000006E
:10029000000000000000000000000000000000005E
:1002A000000000000000000000000000000000004E
:1002B000000000000000000000000000000000003E
:1002C000000000000000000000000000000000002E
:1002D000000000000000000000000000000000001E
:1002E000000000000000000000000000000000000E
:1002F00000000000000000000000000000000000FE
:1003000000000000000000000000000000000000ED
:1003100000000000000000000000000000000000DD
:1003200000000000000000000000000000000000CD
:1003300000000000000000000000000000000000BD
:1003400000000000000000000000000000000000AD
:10035000000000000000000000000000000000009D
:10036000000000000000000000000000000000008D
:10037000ADB200110000000000000000000000000D
:10038000000000000000000000000000000000006D
:10039000000000000000000000000000000000005D
:1003A000000000000000000000000000951AFF1F80
:1003B000000000000000000000000000000000003D
:1003C000000000000000000000000000000000002D
:1003D000000000000000000000000000000000001D
:1003E000000000000000000000000000000000000D
:1003F00000000000000000000000000000000000FD
:081838006071FF1F4118FF1F42
:10184000024981F3088802F02BFC00006071FF1F41
:1018500010B502F02DFB072804D0122808D002286A
:1018600008D010BD044A0420136B01331363F8E75A
:101870000220F6E71420F4E72867FF1FF8B50700F9
:101880000C0026002500503630785135002804D150
:101890000300287058342370F8BD2978CA00481E08
:1018A0008141A3183800A25C5B68C9B2FFF7D0FF82
:1018B00000280DD12B78DA00A218013350602B706C
:1018C0003378044A013B3370136A01331362D8E75B
:1018D0000123DFE72867FF1F5C234343074910B557
:1018E000C9180B0058331B78012B05D1FFF7C6FF31
:1018F000034A936A0133936210BDC0465C67FF1FC1
:101900002867FF1F10B502F023FC064A01211300CF
:1019100010CB4942D967044B136002F059FC2000F8
:1019200010BDC04600E100E01000100010B504003A
:1019300002F00EFC024B1C6002F04AFC10BDC046D7
:1019400000E100E010B5040002F002FC4021094A69
:10195000200013688B43136002F052FB01F0BCFDC2
:101960000022054B01201A60044B04321A6002F079
:10197000D7FAFEE71CF00040C4F00040C0F0004081
:10198000431E5A425341A022F0B5D2015B4213409C
:10199000154D164A40019B182A18127E8BB00191F2
:1019A000002A1BD01A000832D46F0022E6B206AF1C
:1019B000E4B294420EDC2818C369002B08D00199C8
:1019C00002AA117106AA049202AA167303A89847E4
:1019D0000BB0F0BD1978B9540132EAE71A7D1A78D4
:1019E00006AB01261A70E6E7E869FF1F00400040D9
:1019F000F0B5254B04004001C25C85B0002A2BD015
:101A00001A18117E002927D0917E002924D011793F
:101A1000022921D11689D788D168F51BADB22A1CBD
:101A2000102D00D9102292B2BE4217D118180123EE
:101A300003710023C269C38003819A4206D06846BD
:101A4000032103730171029301A890470820002C21
:101A500000D0192001F038FC05B0F0BD013C654212
:101A60006C41A0256442ED012C40084D1B186419FF
:101A7000074D0633013A92B2AA42EDD01888461CAF
:101A80001E80085C2070F5E7E869FF1F00400040F9
:101A9000FFFF00000F220E4B10B59868104002386F
:101AA0000A280BD802F026F90D0A0B0A0A110A0AB5
:101AB0000A0A060002210020FFF762FF10BD012183
:101AC000F9E70020FFF794FFF8E7DB6FF6E7C04681
:101AD000004000400F220E4B10B5986810400238AD
:101AE0000A280BD802F006F90E0A0B0A0A120A0A93
:101AF0000A0A060002210120FFF742FF10BD012162
:101B00000800F9E70120FFF773FFF7E7DB6FF5E760
:101B10000090004013B5334C2378072B3DD8324B4F
:101B20001A78324B002A39D18022196852020A43AE
:101B30001A60252001F08CFF20232D4A11680B43E9
:101B4000802113606B460422C905086807331042E0
:101B500028D080210422C905C86810422ED08021D7
:101B60002020C905CA688243CA6014221A701A78F4
:101B7000002A2FD18021C905C86820320243CA60DB
:101B800014221A701A78002A28D11A4B1A7D22784A
:101B90005A601D221A705932DA6013BD1A6816494C
:101BA0000A40C5E7086802430A6014221A701A78CE
:101BB000002ACED01A78013AD2B2F7E7C8680243B9
:101BC000CA6014221A7019784A1ED2B21A700029FB
:101BD000F9D1C4E71A78013AD2B2C7E71A78013AC4
:101BE000D2B2CEE76045FF1F2846FF1F3CF0004001
:101BF0005845FF1F00200040FFFFFEFF564B70B509
:101C00001B68012B03D1554A936D0133936502F094
:101C1000B7F8534B534A1860534B544C1A60012386
:101C2000534A1360534A13602378002B06D00622D0
:101C30005149524802F00CFA00232370504A514B8C
:101C400010681B78C1B2002B0ED14F4CC0B2237864
:101C50005BB2002B4FDB237824785BB264B21B04A9
:101C600024021B191B1813600B1C50294ED950233A
:101C7000464A47491078DBB2FF2202284BD1086858
:101C8000444C454D267890432A78964254D9227880
:101C900024782E78023B5D10A31B6B435201D31AAC
:101CA00010335B111843086002F0EAF8031F012BA0
:101CB00045D83A4B1B78002B06D0394B1B78002BAC
:101CC00002D0002002F054FAA122364B92009978FB
:101CD000354B4A431B689B18832292009B181B7844
:101CE000033B012B03D8AF20400002F031F9012261
:101CF0002E4BDA8270BD237824785BB264B2FF3356
:101D0000FF341B0424021B190138ABE7CAB2022AB4
:101D1000AED20223ACE70868254C264D26789043C6
:101D20002A78964208D9227824782D78023B5B10D5
:101D3000641B63435201B2E72378DBB2B2E70228A7
:101D4000D5D11D4B1B78013B022B03D91B4B1B78B4
:101D5000022BCCD16C20C8E79809FF1FFC0FFF1F96
:101D60006066FF1FFF3F0000141003406466FF1F02
:101D70000C10034000100340D50BFF1F7211FF1F12
:101D8000B40003408C09FF1F680AFF1F490AFF1FA8
:101D900094000340460AFF1F470AFF1FF908FF1F70
:101DA0002209FF1F300DFF1F3409FF1FBC0BFF1F4F
:101DB000440AFF1F450AFF1F1C09FF1F2309FF1FBD
:101DC00010B502F085F80022014B1A8010BDC04604
:101DD0005C66FF1F10B502F043F9A121054A890096
:101DE0009478054A61431268044B5218528C1A8049
:101DF00010BDC046300DFF1F3409FF1F5C66FF1F7A
:101E000010B50D4B0D4A9978A1239B004B431268E6
:101E1000D218531DD97F0A4B1B88994209D2441C02
:101E200007D0C82805D0D2695B1A5A43054B5343E3
:101E3000C01802F0BDF810BD300DFF1F3409FF1FA0
:101E40005C66FF1F7102000070B5244D2B68002BEB
:101E500028D001F0A5FF2B68D8402B680400002B88
:101E600027D002F02DF82B68D8401D4B1D4A9978D9
:101E7000A1239B004B431268D118D25C91239B0095
:101E8000002A20D0CA580132CA50174B17491B6884
:101E90000868834214D3D23B181A012A1AD0144B73
:101EA000186070BD01F07CFF124B196802F088F8D1
:101EB000D3E702F005F80F4B196802F081F8D4E778
:101EC0000D495B18E8E7CA500C4B1B68DB68E41847
:101ED000201AE4E7F530FF30E1E7C0461C08FF1F99
:101EE000300DFF1F3409FF1F9C09FF1F6066FF1F95
:101EF000A009FF1F1808FF1F2DFF3F006866FF1F86
:101F000070B504000D00282916D10300A433C2883F
:101F10001B889B1A0B4A9BB293420DD906006A3666
:101F200005223100653002F03BF8002804D1310071
:101F3000200001F01DFF70BD2900200002F0A0F874
:101F4000F9E7C046FE7F0000F8B50400012001F06B
:101F50008FFF01F0F5FE194A03001060184E194872
:101F6000016831600568A942FAD11748174E056823
:101F700077680020AF4201D27068281A144D091901
:101F800028601448C162A421446A49032143416284
:101F900011490978002905D010490978022902D190
:101FA0000F3B1360F8BD012901D1083BF9E7032974
:101FB00001D1053BF5E7033BF3E7C046E408FF1F0B
:101FC000340AFF1F28F00040180AFF1F28100040A5
:101FD0001C0AFF1F00F000401C09FF1F4A0AFF1FD8
:101FE00070B580241025E405A3682B43A36001F09D
:101FF000CFFEA368AB43A36070BD0000F7B5160029
:1020000080221C001023D2050191916805000B432A
:10201000936000225A4BD7301A6001F0D1FE9D2305
:102020002A002F009B00EB58CA3201210092FC3796
:10203000002B01D00021009A386802F019F829001D
:10204000009BCB311A784F4BD3351A604B780A7806
:102050001B0213438A7812041A43CB781B061343DE
:10206000494A1BBA13604B790A791B0213438A79D8
:1020700012041A43CB7931001B061343434A1BBA9F
:1020800013606B782A781B021343AA7812041A4350
:10209000EB781B0613433E4A1BBA1360019A3302C6
:1020A00013433C4A13603C4B22001B1B9C460329F4
:1020B0003DDCB3089A0013005142B21A032A46D1FC
:1020C000354AE018511A827840781204000202431F
:1020D000E05C043302430A600022FF2B4BDDF02258
:1020E0002E4B12011A600F222D4B1A602D4A1368D5
:1020F000002BFCD00023224A27491360091B321D04
:102100000B191B68043A180A23706070180C1B0E18
:10211000A070E3700434002AF2DC802210213B68B6
:10212000D20501333B6093688B439360F7BD6346F0
:10213000D578981893782D061B042B43157804390D
:102140002B43557804322D022B430360AFE7022A5C
:102150000AD1114AE05C511AE21852781202024385
:102160000A6004339BB2B7E7012AB5D10A4A521A72
:10217000E15C1160F5E7084959180A600433ACE7DF
:10218000000004403C000440380004403400044097
:10219000300004400C0004400001044004000440EE
:1021A0001000044014000440F7B5150080221C0004
:1021B0001023D2050091916807000B439360002320
:1021C000654AD730136001F0FBFD9D233E009B0064
:1021D000F9583B00CA363200FC33002900D07FE0BA
:1021E000586801F045FF390032785C4BCB311A60FA
:1021F0004B780A781B0213438A78AC4612041A43C0
:10220000CB78281D1B061343554A1BBA13604B7924
:102210000A791B0213438A7912041A43CB791B06ED
:102220001343504A1BBA13604B7A0A7A1B021343BA
:102230008A7A12041A43CB7A21001B0613434A4AB6
:102240001BBA1360009A2B021343484A1360220002
:10225000474B1B1B0093009BCE785B1801938B7838
:1022600036061B0433430E78043833434E7804316A
:1022700036023343019E33600328ECDC0321A808B7
:10228000431C9B002940800003292BD13849E518C5
:102290005E18A9786D78E35C09042D02294319437F
:1022A0003160030008330021FF2B2DDD314B324913
:1022B00019600F21314B1960012327490B60304B06
:1022C00019680029FCD006211B680B40042B20D084
:1022D00080220020D20593680A318B439360FEBDB3
:1022E00001217DE7022908D121495D18E1184978CB
:1022F000E35C090219432960D3E70129D3D11C49C2
:102300005918E35C0B60CCE71948181801600433D6
:10231000CAE7002310490B606346002B0CDC3B002E
:10232000FC335A68102101325A608022D20593682A
:1023300001208B439360D2E7009B9B181B68190A0E
:1023400013705170190C1B0ED37004235B429170F3
:102350009C440432E0E7C046000004403C000440D6
:102360003800044034000440300004400C000440B5
:102370000001044004000440080F00001000044065
:102380001400044070B5061E19D00222614B9B79DF
:102390009343012B13D1604B1A78FF2A0FD15A783F
:1023A000FF2A0CD19A78FF2A09D1DA78FF2A06D1C0
:1023B0001A79FF2A03D15B79FF2B00D1A7E0574B95
:1023C0000C201A78012A08D00022554D1A702B785B
:1023D0001A00093A042A01D8212070BD5A1F012A87
:1023E000FAD94C4CA07B042800D990E0A279032AAA
:1023F00000D98CE0821E012A03D862881F2A00D8E7
:1024000085E0002E61D0012E00D080E0A288012A54
:10241000E2D0002B0AD10138032803D801F06AFC6E
:10242000151D19151F202E7001F08AFD2B785A1EDC
:10243000032A16D800253B4B1D602823237501F085
:1024400047FEA8422ED0A580C6E7022320202B708D
:10245000EAE7042322202B70E6E7032321202B70D8
:10246000E2E7073B012BB7D82F4B1B68DB6A9B06C3
:10247000B2D52E4B1A78002AAED1A27B911E01292B
:1024800001D9002AA8D1022280211A702823284DC0
:1024900089012878237501F033FE8021287889018D
:1024A00001F03EFC0123A380224B1B78002B0AD0B5
:1024B000FA228021204B92001B8809025A431C4BB0
:1024C000187801F055FD002087E701F041FE2B78D8
:1024D000A680073B012B06D918482E7001F0B0FEEC
:1024E0001E2001F02DFD114B114C1A78002A06D048
:1024F00080210022207889011A7001F001FE01F08C
:1025000067FE80212078090201F0FAFDDBE7122046
:1025100063E7C046A60BFF1F6B09FF1F1A09FF1FC9
:102520001C09FF1F4809FF1F6866FF1F2309FF1FC3
:102530001B09FF1F2109FF1F2C09FF1F001000406E
:1025400010B5002901D001F06BFC10BDF7B5604B50
:1025500001919978A1239B004B435E4A06001468C1
:102560001022E418D6235B00E0583623FF33E35CE7
:1025700000279343222B41D1574B0F3A1A60076033
:10258000012501F06DFE019B1880E8235B00E35CF0
:10259000002B01D0B34258DD0023504FFB70AD3308
:1025A000FF33E3581A68002A03D09B88DB439B075C
:1025B0001DD03823FF33E35C002B18D09B235B0036
:1025C000E35C002B13D1D133FF33E35CB3420EDA6B
:1025D000A4235B00E15AE018090A023101F058FC1B
:1025E00023000122FE33013E01351A87FA70E823E9
:1025F0005B00E35C002B2AD0A8B2FEBD03683D005F
:10260000002BBED081880430090A023101F040FC61
:10261000D6235B00E3581F60B2E72300B133BA0052
:10262000FF339858013781880430090A023101F0DC
:102630002FFCE8235B00E35CBB42EEDCE822F61AE9
:10264000ED1800235200A354A6E70027F1E720006D
:1026500001F056FC00281FD0002E1DDD73198826BE
:1026600047190193B600200001F0CAFB5A308000E0
:1026700020184068013581880430090A023101F0D0
:1026800007FC200001F014FDA3590133A351BD4202
:1026900002D0019B9D42E6D1114BE35C002BABD0F5
:1026A00095239B00E35C002BA6D00E4BE15A00293A
:1026B000A2D00D4AA35C994202D90133A3549BE7EF
:1026C00000231A212000A35401F092FD94E7C04694
:1026D000300DFF1F3409FF1F00140340E010FF1FDF
:1026E0005A020000720200005E020000F8B51D4BA5
:1026F0001D4F1A78002A10D1BA7B002A02D101326C
:102700001A7003E0032AFAD0022AF8D001F0E0FCA4
:1027100000220120154B1A70F8BD154B154D1C6891
:10272000154B9E7801232B702878C0B200F0DEFC98
:10273000BB7B002B0BD101F053FBA1239B00734308
:10274000E41883239B00E41823782B70E4E7032B21
:1027500002D101F06DFCF0E70020022BDCD101F08A
:10276000D7FBEAE71C09FF1FA60BFF1F2309FF1F6A
:102770003409FF1F490AFF1F300DFF1FF0B587B056
:102780000EAD2F780FAD2D780593AC46634614003F
:102790000E4D0CAA12782E7803930D9B0092019394
:1027A0002200059B029701F0FBFC2E70012C01D04A
:1027B000042C08D1802206498B889343054A12785D
:1027C000D20113438B8007B0F0BDC0461C09FF1F28
:1027D0006C11FF1F7809FF1F0B001B3B70B5040035
:1027E0003020E02B0DD81300E025493BFF3B9BB286
:1027F000ED00AB4205D8034B200019825A8201F04C
:102800001FFB70BD8410FF1F10B501F0B9FA054B16
:1028100000205B68052B04D9034A5268D20200D419
:10282000980810BD00100040FCE100E070B501F018
:102830008FFC0D4B1B68FC33DC691D6AFFF7E4FF5E
:102840006419844204D2094B01241B68002B07D071
:1028500004220024064B1A70064A936901339361DF
:1028600001F0B6FC200070BD6866FF1F9809FF1FCD
:102870002309FF1FFC0FFF1F70B50C4D2B68FC33A5
:102880005C6A01F065FCFFF7BFFF2B680025FC3395
:102890009B6AE318834204D2054B1B68AB4200D10C
:1028A000051B01F095FC280070BDC0466866FF1F3F
:1028B0009809FF1FD722044B92009B5810B5002B9C
:1028C00000D0984710BDC0460000FF1FF0B587B08C
:1028D00001F09AF9FFF7EEFFCA4BCB4C04931B783B
:1028E000022B45D1C94B1B68186A01F0C1FAC84BCD
:1028F000C84A1A60C84BC94A1A60A022C84B520085
:102900001A60049B187801F053FCC649C64801F0D0
:102910008FFAC649C64801F08BFA1022C54BFF203A
:102920001A60802252031A60802292031A60802269
:1029300012041A6001F01CFC012001F001FCFA20D5
:10294000400001F0F5F9582001F002FBBA4801F00F
:1029500017FB012001F004FB072001F069FC22684D
:10296000B64B1A4084235B001343236007B0F0BDCD
:1029700001F096FAB24E0290322001F079FA3368F3
:102980001B0629D43C2001F073FA0F2001F070FAE5
:102990009C4B1B78012B00D11EE180223368A94D8E
:1029A000134200D0A7E02B68032013432B6001F0F3
:1029B0005FFA01F075FA029B0299C31A5A1E81420E
:1029C00000D81A00A04B1A60904B19681E2353437D
:1029D0009E4A9B18CB618AE701F062FA80239C4AE9
:1029E000DB02116803900B4313602268934B994FED
:1029F0001A40282313432360032001F039FA0320EF
:102A00003D6801F035FA3B680320DB03DB0B0093E4
:102A100001F02EFA3B68ED03DB03ED0BDB0B8E4A76
:102A20000193AB18C22B30D8009B9B18C22B2CD81B
:102A3000019B9B18C22B28D8009B2A009D4200D2E4
:102A40001A00009B9D4200D91D00019B934200D2B9
:102A50001300019A954200D915005B1B122B14D864
:102A60000C22336814209343336033687B4A13404D
:102A7000336001F0FDF908213B682268DB038A43DB
:102A80002260774ADB0B13607FE7032001F0F0F947
:102A90003B68DB03DB0B059301F002FA039B039910
:102AA000C21A531E814200D813006E4A93421BD9AA
:102AB000FF23356869492D0A1D4032686B1C1B06CF
:102AC0000A401B0C134333600C23326800209A43E6
:102AD000083B1343336001F00BFA6348634BA84093
:102AE000984206DCFEF72EFF019B009D0093059B9C
:102AF00095E75F48F6E700235E4F554A3B60802329
:102B00001168DB020B43136080222B680320134300
:102B10002B6001F0ADF93B68052601333B60802353
:102B20002A685B0213432B602268444B03201A403F
:102B3000514B1343236001F09BF90821454B1A6860
:102B40002368D2038B432360454B023900931B68F3
:102B5000D20B4B439A420CD89B1A3B2B0BD82368C1
:102B600046490B4023602B680B402B60444B1A6096
:102B70001FE7D31AF1E7013EF6B2002ED4D1236845
:102B80003E4A134023602B6813402B603B68042BA4
:102B900007D9BFF34F8F3B4B3B4ADA60BFF34F8FF0
:102BA000FEE780222B68032093432B6001F060F93D
:102BB0002268224B03201A4028231343236001F08C
:102BC00057F9244B009A1B68DB03DB0B13600822C8
:102BD00023689343236097E707222C4D2B6813400B
:102BE000012B02D1002001F0E3FAAB68284A022051
:102BF0001340AB6001F03CF98023AA685B001343EB
:102C0000AB60D6E64A0AFF1F5CF000406866FF1F13
:102C1000000003400180063DBC0003403408000072
:102C2000A40003407102000014100040FFFF3F00A9
:102C30002810004000E100E03075000000FEFEFFBB
:102C4000C4F0004044F000405066FF1F72060000D0
:102C500040F0004064F0004091FCFFFFFF00FFFFE8
:102C60005866FF1FE30C0000E88000005F361E007E
:102C700060361E00C444FF1F28000100FFFFFEFF56
:102C80005466FF1F00ED00E00400FA053CF0004030
:102C9000FFFEFFFF694E336888331B6883F30888A3
:102CA00001F026FA00F018FC654B664A1B68934257
:102CB00007D0002001F01CF90221634A13688B43FE
:102CC0001360FFF703FE614B614C1878C0B201F04E
:102CD0008FF90023A3600233A3605E4B01202360C1
:102CE00001F0C6F80323A36001F0DAF8040001F054
:102CF00047F8050001F0D4F8574B186001F080FA4E
:102D0000564B1968621A531EA14200D2130080224A
:102D1000D203934201D39B029B0A3268D16AC9074E
:102D200000D478E04E491C0C09689BB24C435943CF
:102D30002402090A641803274A49FC3293680A6886
:102D400049489B1A494A4A4E12684A499B18414AC7
:102D500034609A183B400193036892089C46019B9B
:102D60000A6063440360042B03D901323B400A60CC
:102D700003600B684049E418200001F021F93F4F3F
:102D80003D493B68C3183B602000019301F048F9BE
:102D90003B4C2068081838492060884205D9019BBF
:102DA00001333B6001F03CF9216001F049F9354BFA
:102DB0001B78002B0ED000F0E3FF3168324B4A1B2A
:102DC0001B6812189A4233D2591A4919091A2F4806
:102DD00001F02EF82E4C237A002B0FD000F0D0FFFC
:102DE0003168E3684A1B1218934224D9591A4919C9
:102DF000091A284801F01CF800232372264B83F39C
:102E0000088801F0E5F8022001F09AF8002001F0AE
:102E10006FF800F0DDFFDC0199000234641A5900FC
:102E2000641A09214B438033CB40A408E41882E79D
:102E3000FA218900CBE71949DBE7C0466866FF1F26
:102E40000C0AFF1FB641210310000040490AFF1F72
:102E500014100040C4090000100AFF1F340AFF1FAD
:102E6000380AFF1F200AFF1F280AFF1F1C0AFF1F26
:102E70004C66FF1F240AFF1F710200006008FF1F3D
:102E80002C0AFF1F1C09FF1FE408FF1F0010004051
:102E9000740BFF1F3C10004000000020DC05000008
:102EA000A022054B92009B5810B5002B01D09847EB
:102EB00010BD01F0B5F9FBE70000FF1FA122054B93
:102EC00092009B5810B5002B01D0984710BD01F01F
:102ED000A7F9FBE70000FF1FA222054B92009B58B9
:102EE00010B5002B01D0984710BD01F099F9FBE710
:102EF0000000FF1FA322054B92009B5810B5002B2A
:102F000001D0984710BD01F08BF9FBE70000FF1FCF
:102F1000A422054B92009B5810B5002B01D0984776
:102F200010BD01F07DF9FBE70000FF1F70B500F058
:102F300027FF514B1860042001F002F801F0F0F86F
:102F40000400C30702D401F0CBF870BD00224B4B44
:102F50001A604B4B1878013804282CD800F0CAFEB0
:102F600003231B1F2700200000F0FAFE0128ECD0ED
:102F7000444C2378042B71D101F06AF9002806D063
:102F800001F006F9582000F0E3FF0223237003202C
:102F900000F0D6FFD9E7200000F00AFFE6E72000A6
:102FA00000F05EFFE2E7200000F0C2FFDEE7200055
:102FB00001F0BEF8DAE700F063FF0500012808D150
:102FC000314B1B78053B012B03D82000FFF768FF2E
:102FD000CEE72C4B1B78022B01D0052B20D1022DE4
:102FE00028D12A4B9B7BAB431CD12000FFF766FF07
:102FF000254B18780128BBD16405B9D42349252273
:103000004B7B034205D1233A13405A4253412633A6
:103010001A000B7D9342ABD9322001F051F8A7E79B
:10302000022D07D1184B1B78052B11D12000FFF77B
:1030300053FFDDE7012D0BD1012B03D12000FFF75A
:1030400059FF95E7062B03D12000FFF761FF8FE7BB
:10305000200001F0E5F8022D8AD1C9E7032B04D145
:103060000B4B987C01F08CF891E7072B8FD1094B23
:10307000987B01F04DF88AE79C09FF1F9809FF1F14
:103080009009FF1F2309FF1F1C09FF1FA60BFF1F2D
:10309000BC0BFF1FD40BFF1FFA210A4B0A4A490041
:1030A0001A640A4A5A500A4A04395A50094A0831DD
:1030B0009A64094A5A50094A5C315A50084ADA66F9
:1030C0007047C0460000FF1F7D27FF1F7928FF1FA4
:1030D0002D28FF1F8523FF1FED26FF1F011EFF1F49
:1030E000D51DFF1F10B500F0EDFD10BD8023F7B515
:1030F0009C46264B264F01932649274A274D284CAC
:10310000284B02281AD1604638600868264E3040A5
:10311000802636033043086001990978002909D1D7
:103120001660224A2A60224A2260E02219689143EE
:10313000A03A1BE08021C9021160F2E766463E60BA
:103140000F68194E3E408027FF023E430E600199F2
:10315000097800290DD1176001280ED1154A2A607F
:10316000154A2260E02219689143C03A0A431A6066
:10317000F7BD802189021160EEE7E0210F4A02438A
:103180002A600F4A22601A688A43F0E74B0AFF1F41
:10319000E0000340D80003409000034000000340DB
:1031A0005000034040000340FFFFE3FF0280063D64
:1031B000804508220180063D80660822008006982E
:1031C00080550822F8B51E4B80261A68002014008E
:1031D0003440324232D11A681A4F32431A60012207
:1031E0003B68063093433B6000F042FE0122164DDF
:1031F0002B681E432E603B680A2613433B608027E2
:10320000BF00124B1B683B4211D1013EF6B2FF2EAC
:1032100009D17E220E4B1C682B68E40B14409343AB
:1032200023432B6005E0082000F022FEE9E7002E92
:10323000EFD180222B68600893432B60F8BDC04615
:10324000C4F000405CF0004018F0004068F000401E
:1032500060F0004010B500F083FF01215820034AC0
:1032600000F0F6FDFFF7AEFF10BDC046600AFF1F7D
:1032700010B578220021034800F032FE00F0B0FFC4
:10328000002010BD7069FF1F70B5040000F060FFE2
:1032900000230C200B4A010059438D18515C002972
:1032A0000DD0A14208D1012300246B7000F0B0FDC5
:1032B00000F08EFF200070BD01330A2BEBD11224E9
:1032C000F6E7C0467069FF1F70B5040000F040FFCC
:1032D000002319001D000D4A1078002806D0A042D6
:1032E0000CD1557001310C320A29F5D1002B0AD1CD
:1032F00000F076FF00F06CFF002070BD5078461E95
:10330000B0411B18EEE700F083FDF3E77069FF1F83
:10331000F7B504000C20002384460E4D0192674649
:103320005F43E85D7E19A04212D000280BD10A4B02
:103330009C4662461B7808331370019B70707C5565
:103340007160B360FEBD01330A2BE8D10320F9E7B9
:103350000720F7E77069FF1F6C69FF1F8020F8B531
:10336000484BC0051B68C1248360474BFF251A6882
:10337000012313434361454BA4001A68444B402189
:103380001A60444B1A68444B1A60444B1A59AA43BA
:103390001A51C52292009E58AE433143802699505F
:1033A0009F583F49F6010F403E439E509E5880274C
:1033B0003602360A3043985080201A5900020A40DB
:1033C00002431A5104341A59364E3F0432408026C3
:1033D0003A431A511A5936061202120A32431A5146
:1033E00008341A5980260A4002431A51C322920017
:1033F0009F58B446AF4337439F509F58294E0F40C4
:1034000007439F509F583740802636043743802615
:103410009F509F5836063F023F0A37439F50C022B5
:103420001F59AF433A431A511A591202120A16434E
:10343000C6221E5192009C58AC4365462C439C50BA
:103440009C5800250C4020439850C72080001A58F3
:10345000154C1140C02212020A431A50134B1B781C
:10346000DB08AB4201DC0020F8BD2378002B06D03E
:10347000A368002B00D0984701350C34EEE71220EA
:10348000F2E7C0465C45FF1F5845FF1FB0F0004003
:103490006869FF1FB4F000406469FF1F00E100E0AD
:1034A000FF00FFFFFFFF00FF7069FF1F6C69FF1F38
:1034B000030010B51F2809D8072200201340072455
:1034C00004490A78A24313430B7010BD0023062061
:1034D000F5E7C0466C69FF1F034A044913680020E2
:1034E0000B4013607047C0461CF00040FFFFC1FF57
:1034F000054B06491B780A6805485B0702401B0B11
:10350000134300200B6070476C69FF1F1CF00040E4
:10351000FFFFC1FF70B50C25FFF7EAFF0A4B1C78CF
:103520000A4BE4086543ED18002C01D1200070BD62
:103530002B78002B06D06B68002B00D09847013CFD
:103540000C3DF1E71220F2E76C69FF1F6469FF1F71
:1035500007B50422074801A900F034F9019B0133A3
:1035600005D18023044ADB0411680B43136000205B
:103570000EBDC0461C18001114F00040F0B5050047
:103580002026184B87B00493049B002B03D11124F1
:10359000200007B0F0BD002102220B000191009134
:1035A000052000F025FC02230F490A681A42FCD1CD
:1035B0000596059C631E0593002CFAD10B4A1368EF
:1035C000002BFCDA0F276F440121380000F008FDC2
:1035D0003B782B42DCD0052000F04AFC049B013BE9
:1035E0000493D1E7FFFFFF0790C8004000C80040E8
:1035F00007B500F0ADFD80220821D205936A019144
:10360000002B01D10739916202210C4A1160019906
:10361000481E01900029FAD1033111600531019152
:103620000199481E01900029FAD11160002B02D1A6
:103630008022D205936200F0CBFD07BD00C00040A0
:10364000F0B52D4C89B02378002B4FD1FEF75AF9F5
:1036500002232A4F03903A681A42FCD12023069392
:10366000069B5A1E0692002BFAD1254E3368002B7A
:10367000FCDA0120FFF782FF011E02D0112009B001
:10368000F0BD030003220190009005AD9F2000F0E3
:10369000AFFB0321280000F0A3FC02233A681A4282
:1036A000FCD120230793079B5A1E0792002BFAD1C7
:1036B0003368002BFCDA0120FFF760FF0028DDD122
:1036C0000398FEF733F9AA786B7811041B020B43B9
:1036D00029780B4363601300113B0A49052B07D877
:1036E00001239340A3600B60012323700020C6E7F1
:1036F00080231B03F6E7C0464445FF1F90C80040E7
:1037000000C800409808FF1F1E4B30B55A68187853
:103710001D4B85B0D31859424B4101210093002322
:1037200000F036FC194B1A4A02259A6300221A65EA
:1037300010325A658022C4219D65164B1648D2026C
:10374000DA6789004258154B80241A4080231B04F5
:1037500013434350642341200393E40500F078F9B8
:10376000402000F075F96562039D6B1E0393002DE8
:10377000FAD103236362FFF73BFFA562FFF760FF07
:1037800005B030BD5045FF1F95FFFEF700C8004053
:10379000050001FF04E100E000E100E0FFFF00FFA1
:1037A00010B5064B18705960FFF7AEFF00211320CB
:1037B000034AFFF7ADFD002010BDC0465045FF1F76
:1037C0000937FF1FF0B5040085B003920291FEF7A0
:1037D00099F8882263035B0B52051A438023DB05AB
:1037E0009D6A8023274F0092BA68002601901B0330
:1037F0009A420CD9F82326001B041E401C4206D016
:103800008022214B52025E6219680A431A60002D21
:103810000BD100F09DFC02221C4B1A608023DB05BB
:103820005A62013A9A6200F0D3FC0023039A934251
:1038300020D1002D0AD100F08BFC144B03221D6017
:103840008023DB055A629D6200F0C2FC8023BA68C7
:103850001B039A4208D9002E06D000220A4B0C49BD
:103860005A621A680A401A600198FEF75FF8002051
:1038700005B0F0BD009A0299D2181278CA540133EB
:10388000D4E7C0464445FF1F00C8004000C00040C8
:10389000FFFFFEFFF0B587B0029103920400FEF730
:1038A00031F8019000F054FC802302250122234EC0
:1038B000DB0535605D629A6200F08AFC204F3B6850
:1038C0002B42FCD120230493049B5A1E0492002B0C
:1038D000FAD11C4D2B68002BFCDA0120FFF74EFEBD
:1038E000002802D0112007B0F0BD2000039A0299F1
:1038F00000F066FC022304003A681A42FCD120233F
:103900000593059B5A1E0592002BFAD12B68002BBC
:10391000FCDA0120FFF732FE051EE3D100F018FCAF
:1039200080230322DB0535605A629D6200F050FC63
:103930000198FDF7FBFFE0B2D5E7C04600C00040AC
:1039400090C8004000C80040F0B5802687B0040051
:10395000FDF7D8FFF605B36A02250393029000F045
:10396000F7FB0123244F3D607562B36200F030FC29
:10397000224E33682B42FCD120230493049B5A1E11
:103980000492002BFAD11E4D2B68002BFCDA01208B
:10399000FFF7F4FD002802D0112007B0F0BD200091
:1039A00000F036FB0223019032681A42FCD120233A
:1039B0000593059B5A1E0592002BFAD12B68002B0C
:1039C000FCDA0320FFF7DAFD041EE5D100F0C0FBAE
:1039D00080230322DB053C605A629C6200F0F8FB06
:1039E000039B002B01D1FFF703FE0298FDF79EFF1A
:1039F0006B461879D1E7C04600C0004090C800402F
:103A000000C8004007B5000201910422000A01A984
:103A1000FFF740FF0EBD000073B5050005240B4AFB
:103A2000A3005B429B1819686B46DE1D300000F056
:103A30002FFB022804D133782B55013CEFD276BD01
:103A4000052CFCD00128FAD10230F8E71409001146
:103A50001F2807D8012380228340D20591680B4399
:103A6000936070473F2808D8012380222038834084
:103A7000D20551690B435361F3E75F28F1D8012365
:103A8000802240388340D205116A0B431362E8E775
:103A90001F2807D8012280218240C9058B689343E3
:103AA0008B6070473F2808D801228021203882404F
:103AB000C9054B6993434B61F3E75F28F1D80122B5
:103AC000802140388240C9050B6A93430B62E8E7C6
:103AD0001F2810D880230200DB05153A1968012A37
:103AE00006D820229143196019680A431A6070476A
:103AF00001228240F6E73F2811D880230200DB052F
:103B0000353AD968032A06D810229143D960D9687A
:103B10000A43DA60EBE7012220388240F5E75F28AC
:103B2000E5D842238022181A413B8340D205516ACE
:103B300099435162516A0B435362D8E710B50400B0
:103B4000012813D1A022184992050B685B015B097B
:103B500013430B60154B164A19681140154A0A4366
:103B60001A60402219680A431A6010BD0028FCD16F
:103B700001000A2000F0ECF821000B2000F0E8F82A
:103B8000C0220A4B920019680A4340211A601A6841
:103B90008A431A60B022044912060B685B015B0974
:103BA00013430B60E1E7C04614F000401CF00040F6
:103BB0007F00FEFF80FD010072B6074A13680133E3
:103BC00013600422054B1A600023054A136080220B
:103BD000D2055360FEE7C0467808FF1FC0F00040E2
:103BE000C4F00040044B054A1A60054B1A600022DD
:103BF000044B1A607047C046140AFF1F841E000061
:103C0000380AFF1FC4F000400023034A1360034A30
:103C10001360034A1360704754F0004040F10040C5
:103C200044F10040002310B5184C8AB00093019372
:103C30002378012B27D06946012000F0E9FA0028FB
:103C400017D1009B12490293019B06AA0393114BC3
:103C500002A81B680493104B1B68059300F098F8AA
:103C600010220E4906A800F09BF9002804D1FF237A
:103C7000237000200AB010BD0123094A074902A899
:103C8000237000F085F80120F4E7C0466C66FF1F42
:103C900010290011082900110C29001120290011F8
:103CA0007066FF1F13B501246946012000F0B0FAC9
:103CB000034B00940193FFF7B5FF200016BDC046EB
:103CC000BB0B000010B5FFF79FFFFFF7EBFF0028CD
:103CD00002D0024B984710BDFEE7C046E1A20000AB
:103CE00002B4714649084900095649008E4402BC95
:103CF0007047C04602B4714649084900095C490052
:103D00008E4402BC7047C04603B471464908400067
:103D10004900095A49008E4403BC70470000000066
:103D200001B40248844601BC604700BF0D52010047
:103D300001B40248844601BC604700BF85120100FF
:103D400001B40248844601BC604700BFBD5C01006D
:103D500001B40248844601BC604700BFCD9E0011FB
:103D600001B40248844601BC604700BF0134010031
:103D700001B40248844601BC604700BF85C1000011
:103D800001B40248844601BC604700BFC95C010021
:103D900001B40248844601BC604700BFDD3F00001B
:103DA00001B40248844601BC604700BFE90B010032
:103DB00001B40248844601BC604700BF09340100D9
:103DC00001B40248844601BC604700BF894400003A
:103DD00001B40248844601BC604700BF855201001F
:103DE00001B40248844601BC604700BFE9F6000008
:103DF00001B40248844601BC604700BF496D010020
:103E000001B40248844601BC604700BFD9B000003D
:103E100001B40248844601BC604700BF21A90000EC
:103E200001B40248844601BC604700BFE9D40000E9
:103E300001B40248844601BC604700BF2D6C0100FC
:103E400001B40248844601BC604700BF116E000007
:103E500001B40248844601BC604700BF016701000D
:103E600001B40248844601BC604700BF053401002C
:103E700001B40248844601BC604700BF01890000CC
:103E800001B40248844601BC604700BFDD0C01005C
:103E900001B40248844601BC604700BFC11501005F
:103EA00001B40248844601BC604700BF156B0100A5
:103EB00001B40248844601BC604700BFE927000006
:103EC00001B40248844601BC604700BF6D0B01008D
:103ED00001B40248844601BC604700BF8D820000E7
:103EE00001B40248844601BC604700BFB70E000021
:103EF00001B40248844601BC604700BF016C010068
:103F000001B40248844601BC604700BF71B00000A4
:103F100001B40248844601BC604700BF19FA0000A2
:103F200001B40248844601BC604700BFA1AF000055
:103F300001B40248844601BC604700BFF53501006A
:103F400001B40248844601BC604700BF1907010064
:103F500001B40248844601BC604700BF79120100E9
:103F600001B40248844601BC604700BFE51201006D
:103F700001B40248844601BC604700BF8B52010077
:103F800001B40248844601BC604700BF8D110100A6
:103F900001B40248844601BC604700BFC56D010002
:103FA00001B40248844601BC604700BFCD4C01000B
:103FB00001B40248844601BC604700BF8937010054
:103FC00001B40248844601BC604700BF090E0000EE
:103FD00001B40248844601BC604700BF79970000E5
:103FE00001B40248844601BC604700BF3D71010036
:103FF00001B40248844601BC604700BF8914010037
:1040000001B40248844601BC604700BFF9A6000025
:1040100001B40248844601BC604700BFA96F01009B
:1040200001B40248844601BC604700BF090E00008D
:1040300001B40248844601BC604700BF75F8000027
:1040400001B40248844601BC604700BFD54401006A
:1040500001B40248844601BC604700BFE94C01003E
:1040600001B40248844601BC604700BFF9ED00007E
:1040700001B40248844601BC604700BF21440000EF
:1040800001B40248844601BC604700BF51B800003B
:1040900001B40248844601BC604700BF8D3800115E
:1040A00001B40248844601BC604700BFB9B20011A8
:1040B00001B40248844601BC604700BF5976010044
:1040C00001B40248844601BC604700BF613701006B
:1040D00001B40248844601BC604700BFA9D8000073
:1040E00001B40248844601BC604700BFDD0A0100FC
:1040F00001B40248844601BC604700BFC9A9000062
:1041000001B40248844601BC604700BFB3520100BD
:1041100001B40248844601BC604700BFC1F70000FB
:1041200001B40248844601BC604700BFBD0B0100DA
:1041300001B40248844601BC604700BFF935010064
:1041400001B40248844601BC604700BF6911010008
:1041500001B40248844601BC604700BF75A9000055
:1041600001B40248844601BC604700BFED6801000D
:1041700001B40248844601BC604700BFED6B0100FA
:1041800001B40248844601BC604700BF4DF90000FD
:1041900001B40248844601BC604700BF6DF60000D0
:1041A00001B40248844601BC604700BF9D6A00001C
:1041B00001B40248844601BC604700BFEDA5000081
:1041C00001B40248844601BC604700BF95730100FA
:1041D00001B40248844601BC604700BF9DA90000AD
:1041E00001B40248844601BC604700BFADAE000088
:1041F00001B40248844601BC604700BF53B90000C7
:1042000001B40248844601BC604700BFC16601009A
:1042100001B40248844601BC604700BFE1AC000025
:1042200001B40248844601BC604700BFE9170100A1
:1042300001B40248844601BC604700BFF90D01008B
:1042400001B40248844601BC604700BFC1A500001C
:1042500001B40248844601BC604700BF01D700009A
:1042600001B40248844601BC604700BFCD0C010088
:1042700002000000EEBB001101000000C0B90011F7
:1042800002000000EABB001101000000B042FF1F65
:1042900002000000C8B9001101000000B463FF1F54
:1042A00002000000E8BB0011030000002863FF1FAC
:1042B0001200000002000000EEBB0011010000002F
:1042C00008BA001102000000EABB00110100000062
:1042D00005BA00110200000012BA0011030000002C
:1042E0006363FF1F02000000E8BB00110300000031
:1042F0007863FF1F02000000EABB0011010000000C
:1043000004BA00110200000010BA001103000000FE
:104310003963FF1F02000000E8BB0011030000002A
:104320005A63FF1F02000000EEBB001101000000F5
:1043300048BA001102000000EABB001101000000B1
:10434000F943FF1F020000005ABA001101000000EB
:1043500043BA001102000000EABB00110100000096
:10436000F843FF1F0200000058BA001101000000CE
:104370008063FF1F02000000EABB00110100000083
:10438000F743FF1F0200000056BA001101000000B1
:1043900033BA001102000000EABB00110100000066
:1043A000F643FF1F0200000054BA00110100000094
:1043B0002EBA001102000000EABB0011010000004B
:1043C000F543FF1F0200000052BA00110100000077
:1043D00029BA001102000000EABB00110100000030
:1043E000F443FF1F0200000050BA0011010000005A
:1043F00024BA00110202020202020000A14B0011C5
:10440000654B00119CBA0011900118001800FFFFC5
:104410000701020304050602010600000000000077
:10442000000000000000000000000000000000008C
:10443000000000000000030002000000EEBB0011BD
:10444000010000001CBB001102000000EABB0011CB
:1044500001000000A844FF1F0200000026BB00115D
:1044600001000000AE63FF1F02000000E8BB001166
:10447000030000001C66FF1F02000000EABB0011E1
:1044800001000000A844FF1F0200000024BB00112F
:1044900001000000B063FF1F02000000E8BB001134
:1044A000030000001466FF1F12000000000100005E
:1044B00000000111FFFF00005048593600000000C5
:1044C0000000000001000000ADBA00110B00050063
:1044D000F7000000B4000028002800283075A00074
:1044E000A000A000A00000080008E001F0001000FB
:1044F000100010001000100010005000500050007C
:1045000010001000D0070000000000000F000100A4
:104510000500307507001000010081FF0000000059
:10452000FF000000B5700011BD6E00114D6C001150
:10453000FFFF0100FF000000D19A00114D9800110B
:104540006597001100000000000000000000080056
:10455000040000003B0001085902E0018821280006
:10456000FF00000002000000EEBB0011010000008F
:10457000B4BC001102000000EABB00110100000001
:10458000E145FF1F02000000E6BB00110100000032
:10459000286AFF1F02000000EABB001101000000B2
:1045A000E045FF1F02000000E4BB00110100000015
:1045B000DE45FF1F02000000EABB00110100000001
:1045C000DC45FF1F02000000E2BB001101000000FB
:1045D000D445FF1F180018000000900102000003DE
:1045E0000202000002000000EEBB0011010000000A
:1045F000C8BC001102000000EABB0011010000006D
:104600002446FF1F02000000E0BB00110000000074
:104610000000000002000000E8BB001103000000E1
:06462000486AFF1F20FFA5
:040000051FFF184180
:00000001FF
